:1075D300758400852ED2852FD3E4F52FF52E303810
:1075E30010E50D852DF0A4252EF52EE5F0352FF5AC
:1075F3002F2290760F303E031275FF22E50E251BD6
:10760300F50EE51F351AF51F93F50D227F82858848
:107613008C8F9295989B9EA1A4A7AAADB0B3B6B93F
:10762300BBBEC1C3C6C9CBCED0D3D5D7D9DCDEE070
:10763300E2E4E6E7E9EBEDEEF0F1F2F4F5F6F7F864
:10764300F9FAFBFCFCFDFDFEFEFEFEFEFEFEFEFE69
:10765300FEFDFDFCFCFBFAFAF9F8F7F6F4F3F2F0A1
:10766300EFEDECEAE8E7E5E3E1DFDDDBD8D6D4D103
:10767300CFCDCAC8C5C2C0BDBAB7B4B2AFACA9A654
:10768300A3A09D9A9794908D8A8784817E7A77743C
:10769300716E6B6865625F5C595653504D4A47443F
:1076A300423F3C393734322F2D2A282624211F1DEF
:1076B3001B1918161412110F0E0C0B0A08070605D6
:1076C30004040302020101000000000000000000A6
:1076D3000001010202030405060708090A0B0D0E47
:1076E3001011131516181A1C1E20222427292B2EBD
:1076F300303335383A3D404245484B4E5154565944
:0C7703005C606366696C6F7275787B7F58
:107E0400D2F4C2F5C2F675840F85F0C8127B5074A3
:107E140003127E53127B407403127E53127B2F1283
:107E24007B2F7403127E53127B2F7402127E531223
:107E34007B2F7428127EBF7406127EBF740E127ECE
:107E4400BF7401127EBF127B407480127EBF22C0B9
:107E540000A2E092F3A2E192F2A2E292F1A2E392F2
:107E6400F0D2F475840F85F0C8C2F47830D8FE855A
:107E7400F0C87830D8FED00022C00075840FA2E488
:107E840092F3A2E592F2A2E692F1A2E792F0D2F482
:107E940085F0C8C2F47830D8FE85F0C87830D8FEB2
:107EA400D00022EF75840FD2F5C2F685F0C8127E99
:107EB4007D127B2F127E53127B2F2275840FC2F505
:107EC400C2F685F0C8127E7D127B2F127E53127B80
:107ED4002F22EF14A2E492E6C2E4D2E7127EBF227C
:107EE400740F127EBF22740D127EBF227F01127E98
:107EF400D678107F20127EA7D8F9227F11127ED661
:0A7F040078107F20127EA7D8F92222
:10749600C293758400D2C2C2C6D2C6C2C4D2C5C205
:1074A600C330C3FD74A0F5C2C2C5C2C330C3FD8ECE
:1074B600C2C2C330C3FD8FC2C2C330C3FD8DC2C2B8
:1074C600C330C3FDD2C4C2C320C4FD127B40D293D5
:1074D60022758400C2C3D2C530C3FD74A0F5C2C2F2
:1074E600C5C2C330C3FD8EC2C2C330C3FD8FC2C284
:1074F600C330C3FDC2C4D2C5C2C330C3FD74A1F537
:10750600C2C2C5C2C330C3FDC2C2C2C330C3FD8539
:10751600C207D2C4C2C320C4FD22D2C2C2C6D2C6CA
:10752600D2C4C2C320C4FD22C293758400D2C2C293
:10753600C6D2C6C2C4D2C5C2C330C3FD74A0F5C28A
:10754600C2C5C2C330C3FD8EC2C2C330C3FD8FC223
:10755600C2C330C3FD8C838D827B80E0A3F5C2C29B
:10756600C330C3FDDBF5D2C4C2C320C4FD127B40C9
:10757600D29322758400C2C3D2C530C3FD74A0F570
:10758600C2C2C5C2C330C3FD8EC2C2C330C3FD8FE3
:10759600C2C2C330C3FDC2C4D2C5C2C330C3FD74A8
:1075A600A1F5C2C2C5C2C330C3FD8C838D82C2C3DE
:1075B60030C3FDE5C2F0A31BBB01F3C2C2C2C33098
:0D75C600C3FDE5C2F0D2C4C2C320C4FD2243
:030003000259633C
:01000B0032C2
:0300130002784A26
:1065BA0075FF0775FFDE75FFAD75840F75E1077509
:1065CA00E21475E34475840F75A43575A50975A69B
:1065DA00BB75A7FF759CFF759D00759EF0759FF8AA
:1065EA0075D8FF75E8FF75F80F75AD0F75840175DD
:1065FA00893075888F75840275893075888F75849E
:10660A000F758A80758C67780874FF000000000097
:10661A0000000000000000D5E0F1D8EDE58C30E77D
:10662A00FB759701758A0043890475840075B71054
:10663A0075840F438901758D02758F01758E0474F7
:10664A0080D5E0FD438902E58930E4FB7597027540
:10665A00840075D10775840075BB0175BA0075BCD5
:10666A00F075C70075C60075C5FF75C4FF75E800EB
:10667A0075840275BB0475BA0075BCF175C60075E0
:10668A00C4FF75E88075840075D48475840175D457
:10669A0084758400C2F8759A47759D1A75F8017554
:1066AA00870075840075B90075A900759100759801
:1066BA005075840175989075840075C04075C30043
:1066CA0075CFC9758400758E107589217588057511
:1066DA008400758A00758BE0758CF4758DE04388AB
:1066EA004075840075C90075CA0075CB0075CC0069
:1066FA0075CD0075840175C91875CA8075CBFB758F
:10670A00CDFB75CC80D2CA75840275C91875CAA624
:10671A0075CBAF75CDAF75CCA6D2CA75840075EFAF
:10672A000275A8AC75B83D75E6B075E71D75F6003B
:10673A0075F741789B760A769C780A789D76067575
:07674A00A8959000007F00FC
:106751007E20E4F0A3DFFCDEFA789B760A789C7653
:0E6761000A789D7606D29375E8FF1275202205
:107AA90075840FD2FD2275840FC2FD22E490FC007B
:107AB900732275840FD2EA2275840FC2EA22758473
:107AC9000FA2EC2275840FD2FC2275840FC2FC220E
:107AD90075840FC2FF2275840FD2FF2275840FA20D
:107AE900FA2275840FA2F92275840FA2DD22A292CF
:107AF9002275840FA2DA2275840FA2DB2275840F06
:107B0900A2D82275840FA2D922000000000000002B
:107B1900000000000000000000000000000000005C
:107B2900000000000022C000C001790878B4D8FE26
:107B3900D9FAD001D00022C000C0E078977605E6D6
:107B490070FDD0E0D00022C000C0E07897760FE643
:107B590070FDD0E0D00022C000C0E078977664E6DE
:107B690070FDD0E0D00022EF75F0648424309000DD
:107B790054F0E5F0A375F00A842430F0A3E5F0246D
:107B890030F022EF75F064842430900054F0E5F071
:097B9900A375F00A842430F0A366
:107BA200E5F02430F0900054E0B4300B7420F0A3E0
:107BB200E0B430037420F02275F06484F6E5F00836
:107BC20075F00A84F608A6F00822850607222285A7
:037BD20005062283
:101A1A00C0D0C000C001C083C082C0E0C0F0C0070F
:101A2A00A291304F01B37825E233F208E233F2088B
:101A3A00E233F208E233F208E233F208E233F20860
:101A4A00E233F208E233F208E233F208E233F20850
:101A5A00E233F208E233F208E233F208E233F20840
:101A6A00E233F208E233F208E233F208E233F20830
:101A7A00E233F208E233F208E233F208E233F20820
:101A8A00E233F208E233F208E233F208E233F20810
:101A9A00E233F208E233F208E233F208E233F20800
:101AAA00E233F208E233F208E233F208E233F208F0
:011ABA00E249
:101ABB0033F208E233F208E233F208E233F208E2DF
:101ACB0033F208E233F2305B32784CE218203C03FD
:101ADB0030E728E21820E723E21830E71EE218204F
:101AEB00E719E21830E714E21830E70FE21820E7A5
:101AFB000AE21820E705E21830E703021C5E754086
:101B0B0000E2183392475003754038752200E218F3
:101B1B00339214500363401CE21833921350036347
:101B2B00400EE2183392125003634046E218339290
:101B3B00115003634023E218339210852241500366
:101B4B00634051752200E2183392145003634068CE
:101B5B00E2183392135003634075E218339212501C
:101B6B000363407AE218339211500363403DE2184D
:101B7B00339210852242500363401F752200E218F6
:101B8B00339217500363404FE2183392165003639E
:101B9B004026E2183392155003634052E2183392F9
:071BAB00145003634029E21E
:101BB200183392135003634015E218339212500304
:101BC20063400BE2183392115003634045E218332D
:101BD20092108522435003634062E21833921450FC
:101BE20003634031E2183392135003634019E21841
:101BF200339212500363400DE21833921150036383
:101C02004007E21833921085224450036340437523
:101C12002200E218339216E218339215E218339238
:101C220014E218339213E218339212E2183392112B
:101C3200E218339210852245E5456540701EA247A1
:101C4200924890004DE541F090004EE542F0900040
:101C52004FE543F0900050E544F0D24A121C72D096
:101C620007D0F0D0E0D082D083D001D000D0D022F3
:101C7200C0D0C000C0E0303F4EE552B40833A242AB
:101C8200B392B3787BE66036167880E6A2E73044FA
:101C920001B3924292B2A2E7787CE633F6787DE60F
:0C1CA20033F6787EE633F6787FE633F602
:101CAE007880E633F6D55203755208D0E0D000D0D6
:101CBE00D022C257D0E0D000D0D022D0E0D000D079
:101CCE00D022C0D0C000C001C083C082C0E0C0F02E
:101CDE00A291204E01B3780DE213F208E213F2083E
:101CEE00E213F208E213F208E213F208E213F2082A
:101CFE00E213F208E213F208E213F208E213F2081A
:101D0E00E213F208E213F208E213F208E213F20809
:101D1E00E213F208E213F208E213F208E213F208F9
:101D2E00E213F208E213F208E213F208E213F208E9
:101D3E00E213F2901E85780DE2089313920FE208DB
:101D4E009313920EE2089313920DE2089313920CE2
:081D5E00E2089313920BE20866
:101D66009313920AE20893139209E20893139208D6
:101D7600852146E2089313920FE2089313920EE22E
:101D8600089313920DE2089313920CE208931392B0
:101D96000BE2089313920AE20893139209E208935E
:101DA600139208852147E2089313920FE2089313D2
:101DB600920EE2089313920DE2089313920CE20836
:101DC6009313920BE2089313920AE2089313920973
:101DD600C208852148305B3DE5469021D5854721DF
:101DE600300E02058393602D14F875F003A490203D
:101DF600862582F582E5F03583F583E493F9A3E43D
:101E060093901F85654893C965479329B40100508F
:101E1600048834D241121E2DD0F0D0E0D082D08377
:101E2600D001D000D0D022303D27C392B27881169F
:101E3600E6701E76087884E6A2E1304501B392B3D7
:101E4600A2E17882E613F67883E613F67884E61341
:101E5600F622EF90208575F003A42582F582E583AE
:101E660035F0F583C23D7400937882F67401937859
:101E760083F67402937884F6C23FC23ED23D2200B6
:101E8600000000000000000000000000000000004C
:101E9600000000000000000000000000000001003B
:101EA600000000000000000000000000000001002B
:101EB6000000000000000100000001000101010017
:101EC600000000000000000000000000000001000B
:101ED60000000000000001000000010001010100F7
:101EE60000000000000001000000010001010100E7
:101EF60000000100010101000101010101010100D1
:101F060000000000000000000000000000000100CA
:101F160000000000000001000000010001010100B6
:101F260000000000000001000000010001010100A6
:101F36000000010001010100010101010101010090
:101F46000000000000000100000001000101010086
:101F56000000010001010100010101010101010070
:101F66000000010001010100010101010101010060
:101F7600010101010101010101010101010101004C
:101F8600010102010202030102020302030304012A
:101F9600020203020303040203030303030405010D
:101FA60002020302030304020303040304040502FA
:101FB60003030403040405030404040405050601DD
:101FC60002020302030304020303030304040502DB
:101FD60003030403030405030404050405050602BC
:101FE60003030403040405030404050405050603AA
:101FF600040405040505060405050605060607018D
:102006000202030203030402030304030404050299
:10201600030304030404050304040504050506027A
:102026000303040304040503040405040505060369
:10203600040405040505060405050605060607024B
:102046000303040304040503040405040505060349
:10205600040405040505060405050605060607032A
:102066000404050405050604050506050606070419
:10207600050506050606070506060706070708FD01
:10208600D00C73700E3CF01AAF101E7F9022EC70CD
:1020960026D6F02ACBB02CA3F032BEB03417D03CF3
:1020A600B6D0461FB04E77F050F950526AB056DEA1
:1020B6009058BA306ACF3072D270745CD076E8F03D
:1020C600786BD098E5709AF8309CBB50A40F70AA34
:1020D6007A70B26730B45DB0B8FCB0C26F50C65506
:1020E600D0CA3D90D489B0DA94F0DCD790E463B0DE
:1020F600EA0BF0F43170F8DD310AB571148FF1187E
:10210600D1D126EB512AF6112C8B71463F5148B19D
:10211600F14AACB14CC4F152D9B1546D915A2EF179
:1021260062BD116687916A9AD16CF29172D5517827
:1021360019F18C71B192D8D19A32D1AA47D1B25A3B
:1021460091B452F1C67531CC1D71D2A951DCD0B112
:10215600E85E11EA2B11F2EED212F392147D3216DA
:10216600973226D8B232C5F234F7124AEA524C9F59
:102176005254A5D2582B725A7552644FD268C17206
:102186006ADC326C78D2865F128C83729C4EB2A661
:102196006972AC1C72B433D2CC18F2EABB330CCEE3
:1021A60033141EB32803F32EE51332F85334987311
:0D21B6005848F36472736845738617B3943C
:1021C3007313A63C93B221D3B41B53B829B3C641AE
:1021D300F3D8000000000000000000000000000031
:1021E3000000000000000000006A00000000000082
:1021F300620D0000000000000000006F00480000B6
:1022030000000000000000000000000000006C223D
:1022130000000000000000000000000000000000BB
:102223005B00000000000000000000004100001EF1
:102233004759000000260000001D00001000003573
:102243000000003D006B0043000000000000004B55
:10225300000500000000000000380023000000001B
:102263000000000000000000004C0000000000001F
:102273000000000000000000000000000000320029
:10228300000400000000000000000000126000379E
:102293000A00000000000000000000000008000029
:1022A300611346000000000000254D34000057294B
:1022B30011000000000000640000000000000000A6
:1022C300000000003A4A00002E4F190000001F00D2
:1022D3000000000000630000000000000027000071
:1022E300001B000000000000000B5F3C006E5D441B
:1022F3000000006D0000000000000000005300001B
:10230300360000283F5E00000000000000000300CC
:10231300003000700000006900406700000000000A
:1023230000550000420000210000000000001500DD
:1023330000000000000000000000005C0017000027
:102343000020000068020054000E58001C0000002A
:1023530000000000005A000000000000002F0000F1
:10236300002B00000000240000006600390000007C
:102373000051000000090052000000450000000069
:10238300000000310000002A0C000000001A0000C9
:10239300000000560000334E000000000000000063
:1023A3000000002C1400003B07003E00000000006A
:1023B300000000000000001800001600502D060069
:1023C30049000000000000000000650F000000014C
:1023D30000000000000000000600000006000600E8
:1023E30005020600060006000404060005040208B0
:1023F30006000000060006000600060004080600AA
:102403000600060005080600060002100600060086
:102413000301000006000600020206000600044055
:10242300060006000410060006000600060006006B
:10243300060006000510060006000600060006005A
:10244300060001010600060006000600030206005E
:10245300060000000600060005010600040202044F
:102463000600060006000600060006000600060039
:102473000480060002010420060006000600060090
:102483000600060006000600060006000600060019
:10249300060006000600040106000600060006000A
:1024A30006000310060006000600060006000600EC
:1024B30006000600060006000600060003080600E4
:1024C30006000600060003040600060006000600D8
:0224D300060001
:10596300758400C2CA85CC3885CD3775CC0075CD1A
:1059730000D2CA10CF02D25A32305A0BC25AE5377C
:10598300C394364002800122788C798A7B06E7F63D
:105993001819DBFAA63718A638AA38AB37AE02AF08
:1059A30003EEC4035407FEEFC403FF54F84EFEEFA7
:1059B3005407FF78037987C3E79AFC09E79BFD093E
:1059C30050066304FF6305FFC3EC9EED9F5074D83C
:1059D300E6789479927C06E7F61819DCFAA60318A0
:1059E300A602798FAE02AF03EEC423541FFEEFC4A9
:1059F30023FF54E04EFEEF541FFF7803C3E79AFCE6
:105A030009E79BFD0950066304FF6305FFC3EC9E92
:105A1300ED9F502FD8E6788D7A007B007C007904C7
:105A2300EA26FA08EB36FB08EC3400FCD9F2EC1357
:0D5A3300FCEB13FBEA13FAEC13EB13F53652
:105A4000EA13F535D23A22303A31C23A125A7C5032
:105A50002A853C3D853B3C853A3B85393A8507396B
:105A6000303913E53F6F600EE507B53A0EB53B0BD5
:105A7000B53C08B53D0585073ED23B22905B97E5D6
:105A80003693FF905AC323232582F582E5833400A1
:105A9000F583125AA2400A0F125AA240040F125A5A
:105AA000A222E493F9A3E493FAA3E493FBA3E4937F
:105AB000FCA3C3E5359AE536995007C3EC9535EB61
:105AC000953622EA25DD89DD89D324D324CBD2CBB8
:105AD000D2C4DBC4DBBE39BE39B7CAB7CAB18EB1D6
:105AE0008EAB87AB87A59CA59CA000A0009A969A38
:105AF0009695D895D891E591E58D858D8588AF8867
:105B0000AF840C840C7F9A7F9A7B497B49771B7703
:105B10001B730F730F6F276F276B576B5767AB673D
:105B2000AB642C642C60C660C65D795D795AFE5A00
:105B3000FE5970597057E257E25661566154E75466
:105B4000E7537453745207520750A050A04F404F70
:105B5000404DE64DE64C934C934B414B4149F54942
:105B6000F548B548B547764776463E463E45084532
:105B700008432A432A40E440E43F533F533E3E3E1D
:105B80003E3C943C943A863A8639183918380500D8
:105B90000000000000000032323232323232323243
:105BA00032323232323232323232323232323232D5
:105BB00032323232323232323232323232323232C5
:105BC00032323232323232323232323232323232B5
:105BD000313130302F2E2D2D2D2C2C2B2A292928F8
:105BE00027262525242323222120201F1E1E1D1C9D
:105BF0001C1B1A1A1A1A1919191818181717171717
:105C0000161616161515151514141414131313134C
:105C1000121212121111111110101010100F0F0F7B
:105C20000F0F0E0E0E0E0D0D0D0D0C0C0C0C0B0BA4
:105C30000B0B0B0B0A0A0A0A0A09090909090908C8
:105C400008080808080707070707070606060606E4
:105C500006060505050505050404040404040403FB
:105C60000303030303030202020202020201010111
:105C70000101010101010101010101000000000019
:105C80000000000000000000000000000000000014
:075C9000000000000000000D
:1071EB00C007C0007F01127ED67F4C127EA77F5452
:1071FB00127EA77F52127EA77F20127EA720490402
:10720B007F3080027F31127EA77F20127EA79001F4
:10721B0091E0784B127BC2784B8607430730127E86
:10722B00A7088607430730127EA7750720127EA793
:10723B00900192E0784B127BBA784B86074307306C
:10724B00127EA7088607430730127EA708860743DE
:10725B000730127EA7750720127EA7900193E07866
:10726B004B127BC2784B8607430730127EA70886EA
:10727B0007430730127EA7750720127EA7D000D0D8
:10728B000722C007C0007F11127ED67F4C127EA74B
:10729B00750720127EA7204D047F3080027F3112AC
:1072AB007EA77F20127EA790015BE0784B127BC2FA
:1072BB00784B8607430730127EA7088607430730B3
:1072CB00127EA7750720127EA790015CE0784B1207
:1072DB007BBA784B8607430730127EA70886074395
:1072EB000730127EA7088607430730127EA7750763
:1072FB0020127EA790015DE0784B127BC2784B8603
:10730B0007430730127EA7088607430730127EA774
:10731B00750720127EA790015EE0784B127BC27836
:10732B004B8607430730127EA708860743073012A8
:07733B007EA7D000D007225D
:106F2D00003800512372461765340E5F2D7C4819C9
:106F3D006B3A1C4D3F6E5A0B792812433160540544
:106F4D007726001F3D227A654758756A48570F10FE
:106F5D00322D6877554A120D2F301D02203F67786C
:106F6D005A45006245270B694E2C157750321E7C11
:106F7D005B39294B6C0E224067053C5E791B3755FA
:106F8D00721052301775593B1C7E472502604C2EEE
:106F9D00096B7B193E5C701235576E0C2B496507DA
:106FAD002042264463012D4F680A33517614385A16
:106FBD007D1F0F6D4A28046641231A785F3D1173BA
:106FCD005436741631537F1D3A58610324466A08AE
:106FDD002F4D5D3F187A56341371482A0D6F43219A
:106FED0006644F2D0A68442601635A381F7D5133BC
:106FFD001476660423416D0F284A73113654781A9E
:10700D003D5F1D7F583A16745331086A4D2F036149
:10701D004624345671133F5D7A18214364062A487D
:10702D006F0D690B2C4E620027457C1E395B771561
:10703D003250402205674B290E6C553710725E3C5D
:10704D001B793B597E1C305275172E4C6B09254709
:10705D00600212705735197B5C3E076542200C6E3D
:10706D00492B004307440D4E0A49195A1E5D14570A
:10707D001350317236753C7F3B78286B2F6C25662B
:02708D0022617E
:10869300788076ACA24DE433FFC4333354C0FE90EC
:1086A300015DE0FD541F25E04EFE90015BE0FC54AC
:1086B30010C4540F4E787FF6EC540FC454F0FE9060
:1086C300015CE0FC54F0C4540F4E787EF6EC540F7A
:1086D300C454F0FE90015EE0FC541EC3134E787D3B
:1086E300F6EF3395E0FE742D2FF582746F3EF5831C
:1086F300E493FFED906F2F93FEEF6EFF90015BE02D
:10870300906F4F936FFF90015CE0906F6F936FFFDB
:10871300EC90706F936F787CF690015EE030E0042C
:0B872300E64480F6D257787B762822CF
:10924B00758401309914C29920500F900159E07028
:10925B0009D250D29C789576042230983790015AD7
:10926B00E06401702DE54975F0058420551124EF5C
:10927B00F582E43400F583E599F0C298D2552224A7
:10928B0004F582E43401F583E599F0C298C255D216
:05929B005622C29822DA
:108206007584012098030282CC205213209A0DE532
:10821600997009D252D253754A0AF549C2982290EA
:10822600015AE0FF6401702CE54975F0058420557C
:108236001024EFF582E43400F583E599F0D25580F9
:10824600102404F582E43401F583E599F0C255D291
:1082560056C29822EFB4021AAB530555E555AA54F7
:108266007002055414F9E59912863390015A740385
:10827600802090015AE0FFB4031CAB530555E55529
:10828600AA547002055414F9E59912863390015ADE
:108296007404F0C29822EFB4042990018CE0FF0424
:1082A600F074632FF582E43401F583E599F0C29802
:1082B60090018CE0B4281C90018E7401F0E49001CA
:1082C6005AF022C2982230990AC299900159E07058
:0482D60002C2552269
:1099FA00205122127ADF43E740754A0AE4F549907A
:109A0A000159F090015AF0C250D2517584017598EB
:069A1A0090C29CF59922A8
:1090210090018DE0705C9001ABE0FF7025D3900161
:1090310060E0948690015FE094674008E4F0A374D7
:1090410002F0800E900160E02428F090015FE0348E
:1090510000F0900160E02FFF90015FE03400FE120C
:1090610074D79001ABE02463F582E43401F583EF1A
:10907100F09001ABE004F0E0B42807E4F090018D3A
:0390810004F022D6
:108B9D0090018EE0607A900161E0FEA3E0FFC39446
:108BAD0002EE94005006E490018EF0229001ABE0AD
:108BBD007C002FFFEC3EFE1274D79001ABE02463D6
:108BCD00F582E43401F583E0FD6F60179001ABE0B1
:108BDD00FF900162E02FFF900161E03400FE1274FE
:108BED0096D2549001ABE004F0E0B42823E4900158
:108BFD008EF09001ABF0900161E07004A3E064028F
:108C0D00700E30540BC2541288591290E4129140D8
:018C1D002234
:108EEC003050647584019001A0E0B40D0050559091
:108EFC008F02F8282873028F29028F2C028F2F02E1
:108F0C008F32028F35028F38028F3B028F3E028FD9
:108F1C0041028F44028F47028F4A028F4D029947BC
:108F2C00029B5C0294B60296B9029A2002005E0281
:108F3C0098E30298100296F50294F9029AFB0299B2
:088F4C00A2029AE0129B15221B
:109947007895E67028759898754A0AF54990005BEE
:10995700E0B401079001A07404F022E490015AF0EA
:0E996700900159F09001A0E004F0127AD9228C
:109B5C0090015A7401F0E4900159F0C2559001A0A3
:049B6C00E004F022FF
:1094B60090005BE01475F005A4B54919E4B5F01504
:1094C600759898127ADFE4900159F090015AF0905D
:1094D60001A07404F0E54975F00584AFF0BF0112F0
:1094E600C256E4900159F090015A04F09001A0E0B0
:0394F60004F0225D
:1096B900E54975F00584AFF0BF043020561EE54931
:1096C90075F00584FF24EFF582E43400F583E4F0B6
:1096D90074042FF582E43401F583E4F0E490015930
:0C96E900F090015AF09001A0E014F02273
:109A200090005BE075F005A424FDB5491590005247
:109A3000E0F599E4900159F090015AF09001A0E00E
:039A400004F0220D
:0D005E00900053E0F5999001A0E004F0221D
:1098E30090005BE0FD75F005A4FFE549B50723E4AF
:1098F300B5F01FEDB414079001A07409F022127A99
:10990300D9E4900159F0C25590015AF09001A0E0BA
:0399130004F0223B
:10981000E549B46412127ADFE4900159F090015ADC
:10982000F09001A07409F0E54975F00584AFF0BF30
:109830000112C256E4900159F090015A04F09001CF
:05984000A0E004F0228D
:1096F500E54975F00584AFF0BF043020561EE549F5
:1097050075F00584FF24EFF582E43400F583E4F079
:1097150074042FF582E43401F583E4F0E4900159F3
:0C972500F090015AF09001A0E014F02236
:1094F900E5496465703C90018DE0B4012F75530115
:1095090075540175555FE4900159F090015AF07551
:109519008401AB530555E555AA547002055414F955
:109529001285EDF5999001A0E004F0229001A07454
:039539000CF02211
:109AFB00758401AB53AA54A9551285EDF599E490E1
:0A9B0B00018BF09001A0E004F022AD
:1099A20075840190018BE0FF04F074632FF582E46B
:1099B2003401F583E0F59990018BE0D39428400BB4
:0C99C200E490018DF09001A0E004F02280
:109AE000E549B46915C250C251E49000EDF090010F
:0B9AF00059F090015AF09001A0F02204
:109B1500C250C251E4F5499000EDF0900159F09022
:089B2500015AF09001A0F022AA
:1091F5003052527584019001A1E0B40A00504390A9
:10920500920BF828287302922902922C02922F02BF
:10921500923202923502923802923B02923E0292BB
:10922500410292440297DA02973102976A029AA3A1
:10923500029BCC0299CE0295C10297A2029A4302E3
:069245009BBB129BDC2222
:1097DA00E549703175989890005BE0B40113127AEC
:1097EA00DFE490015AF0900159F09001A17403F05E
:1097FA0022127AD9C255E490015AF0900159F09098
:06980A0001A1E004F022C0
:1097310090005BE01475F005A4B54911E4B5F00D96
:10974100759898127ADF9001A17403F022E54975AA
:10975100F00584AFF0BF0110C256C25590015A7492
:0997610001F09001A1E004F022E6
:10976A00E54975F00584AFF0BF042C20561EE54983
:10977A0075F00584FF24EFF582E43400F583E4F004
:10978A0074042FF582E43401F583E4F0E490015A7D
:08979A00F09001A1E014F0229F
:109AA30090005BE075F005A424FDB54911758401B0
:0F9AB300900052E0F599C2559001A1E004F02215
:109BCC00758401900053E0F5999001A1E004F02216
:1099CE0090005BE0FFB414079001A17406F022EF43
:1099DE0075F005A4B54914E4B5F010127AD99001CA
:0C99EE00A1E004F0C255E490015AF02200
:1095C100E54975F00584AFF0BF0111C256C255904F
:1095D100015A7401F09001A1E004F022E549B4645C
:1095E1001F127AD990018EE0700B90015AF0900110
:1095F100A17408F022E490015AF09001A17409F0DD
:019601002246
:1097A200E54975F00584AFF0BF042C20561EE5494B
:1097B20075F00584FF24EFF582E43400F583E4F0CC
:1097C20074042FF582E43401F583E4F0E490015A45
:0897D200F09001A1E014F02267
:109A4300E549B4651A755301755401755561E49080
:109A5300018CF09001A17409F090015A7402F02274
:109BBB00E549B4690BC252E490015AF09001A1F04F
:019BCB002277
:109BDC00C252E490015AF0900159F09001A1F02288
:1082DA007898E6600116900000E0600214F09000C1
:1082EA0001E0600214F0900002E0600214F09000D5
:1082FA000BE0600214F090000AE0600214F0789A31
:10830A0016E660030283AD789A760A7899E66001E8
:10831A0016900004E0600214F0900005E060021478
:10832A00F0900006E0600214F0900008E060021489
:10833A00F0900009E0600214F0789EE66001169061
:10834A000003E0600214F09001E7E0600214F078A4
:10835A009B16E6704E789B760A90000CE060021439
:10836A00F078A0E61846600708E61618700116901D
:10837A0001A3E0600214F09001A4E0600214F090FE
:10838A0001A7E0600214F0789C16E67016789C76D5
:10839A000A789D16E6700C789D76069001A6E06034
:0483AA000214F022A7
:106AC400535155452020434F53202053454E5345A1
:106AD400004F4E2020202020202020202020202075
:106AE40020004F4646202020202020202020202047
:106AF4002020002020205245504541544552203149
:106B04002020200020202052455045415445522049
:106B14003220202000202020524550454154455227
:106B24002033202020002020205245504541544548
:106B3400522034202020002020205245504541542A
:106B44004552203520202000202020524550454128
:106B54005445522036202020002020205245504504
:106B640041544552203720202000202020524550F7
:106B740045415445522038202020002020205245F1
:106B840050454154455220392020200020202052D5
:106B940045504541544552203130202000202020CA
:106BA4005245504541544552203131202000202087
:106BB4002052455045415445522031322020002076
:106BC4002020524550454154455220313320200065
:106BD4002020205245504541544552203134202034
:106BE4000020202052455045415445522031352043
:106BF4002000202020524550454154455220313632
:106C04002020002020205245504541544552203137
:106C14003720200020202052455045415445522021
:106C240031382020002020205245504541544552FF
:106C34002031392020002020205245504541544520
:076C44005220323020200035
:10002E00750C01E50CC394155018AF0C74182FF510
:10003E0082E43401F583E0FFEF60037F0122050CBB
:04004E0080E17F00CE
:01005200228B
:10919C0020575512847CEF6401704D90009AE0FFCB
:1091AC00EF24FF924D900158E0FF74422FF582E4BA
:1091BC003401F583E0FF90015BEFF0900158E0FF84
:1091CC00742D2FF582E43401F583E0FF90015CEF00
:1091DC00F0900158E0FF90015DEFF01264049001F3
:0991EC005EEFF0128693D23F22DF
:10847C009000E8E4F0A3E4F09000EBE4F0A3E4F067
:10848C009000E7E4F09000E7E0FFEFC394154003A1
:10849C00028520900158E0FFEFD394144006900120
:1084AC00587401F0900158E0FF74182FF582E434F1
:1084BC0001F583E0FF9000EAEFF09000EAE0FFEFB7
:1084CC00B40115900158E0FF74182FF582E43401C3
:1084DC00F5837402F07F01229000EAE0FFEFB40212
:1084EC00249000E8E0FEA3E0FFEF4E70189000E847
:1084FC00E4F0A37401F0900158E0FF7E009000EBD3
:10850C00EEF0A3EFF0900158E004F09000E7E004E7
:10851C00F00284919000E8E0FEA3E0FFEF4E7004BF
:10852C007F0022229000ECE0FF900158EFF07F01D9
:01853C00221C
:1083AE009000E8E4F0A3E4F09000EBE4F0A3E4F036
:1083BE009000E7E4F09000E7E0FFEFC39415400370
:1083CE0002845F900158E0FFEFD3941440069001B1
:1083DE00587401F0900158E0FF74182FF582E434C0
:1083EE0001F583E0FF9000EAEFF09000EAE0FFEF86
:1083FE00605090005BE0FF900158E0FEEE6F60422F
:10840E009000EAE0FFEFB40115900158E0FF7418F8
:10841E002FF582E43401F5837402F07F012290007F
:10842E00E8E0FEA3E0FFEF4E7018900158E0FF7EEB
:10843E00009000EBEEF0A3EFF09000E8E4F0A374F0
:10844E0001F0900158E004F09000E7E004F00283A0
:10845E00C39000E8E0FEA3E0FFEF4E70047F002221
:0E846E00229000ECE0FF900158EFF07F012219
:1064040090005BE0FFEFD3941440037F20229001BF
:10641400EDE4F09001ECE4F090005BE0FF9001EA21
:10642400EFF0900095E0FFEFD3940650030264F878
:106434009001EBE4F09001EBE0FFEFC3941540030F
:106444000264F19001EAE0FFEFB415069001EA74EA
:1064540001F09001EAE0FF74EE2FF582E43400F5D8
:1064640083E0FFEF64FF70769001EAE0FF74BE2FD3
:10647400F582E43400F583E0FF90005BE0FE74BE37
:106484002EF582E43400F583E0FEEEC39F404F9086
:10649400005BE0FF9001EAE0FEEEB507069001EA3A
:1064A400E0FF229001EAE0FF74BE2FF582E434009D
:1064B400F583E0FF9001ECE0FEEFD39E40209001D5
:1064C400EAE0FF9001EDEFF09001EAE0FF74BE2FE7
:1064D400F582E43400F583E0FF9001ECEFF09001E5
:1064E400EBE004F09001EAE004F00264399001ED7D
:1064F400E0FF22229001EBE4F09001EBE0FFEFC318
:10650400941540030265B49001EAE0FFEF70069031
:1065140001EA7414F09001EAE0FF74EE2FF582E4CE
:106524003400F583E0FFEF64FF70769001EAE0FF4A
:1065340074BE2FF582E43400F583E0FF90005BE045
:10654400FE74BE2EF582E43400F583E0FEEEC39FB4
:10655400404F90005BE0FF9001EAE0FEEEB50706D5
:106564009001EAE0FF229001EAE0FF74BE2FF58279
:10657400E43400F583E0FF9001ECE0FEEFD39E40AD
:10658400209001EAE0FF9001EDEFF09001EAE0FFD6
:1065940074BE2FF582E43400F583E0FF9001ECEF44
:1065A400F09001EBE004F09001EAE014F00264FDE5
:0565B4009001EDE0FF85
:0165B90022BF
:1069240090005BE0FFEFD3941440037F202290019A
:10693400F1E4F09001F0E4F0900095E0FFEFD394DF
:10694400065003026A0990005BE0FFEF04FF900128
:10695400EEEFF09001EFE4F09001EFE0FFEFC3946D
:10696400154003026A029001EEE0FFEFD394144055
:10697400069001EE7401F09001EEE0FF74EE2FF545
:1069840082E43400F583E0FFEF64FF70629001EE6F
:10699400E0FF74BE2FF582E43400F583E0FF90003D
:1069A4005BE0FE74BE2EF582E43400F583E0FEEE77
:1069B400C39F403B9001EEE0FF74BE2FF582E434A8
:1069C40000F583E0FF9001F0E0FEEFD39E402090BD
:1069D40001EEE0FF9001F1EFF09001EEE0FF74BEF4
:1069E4002FF582E43400F583E0FF9001F0EFF0909E
:1069F40001EFE004F09001EEE004F002695C900124
:106A0400F1E0FF222290005BE0FFEF14FF9001EE23
:106A1400EFF09001EFE4F09001EFE0FFEFC3941585
:106A24004003026ABE9001EEE0FFEF70069001EEB3
:106A34007414F09001EEE0FF74EE2FF582E434005C
:106A4400F583E0FFEF64FF70629001EEE0FF74BE37
:106A54002FF582E43400F583E0FF90005BE0FE74E0
:106A6400BE2EF582E43400F583E0FEEEC39F403B86
:106A74009001EEE0FF74BE2FF582E43400F583E06C
:106A8400FF9001F0E0FEEFD39E40209001EEE0FF86
:106A94009001F1EFF09001EEE0FF74BE2FF582E477
:106AA4003400F583E0FF9001F0EFF09001EFE00493
:0F6AB400F09001EEE014F0026A1B9001F1E0FF98
:016AC30022B0
:10676F0090005BE0FFEFD3941440037F2022900052
:10677F0052E0FFEFB4FF0C900053E0FFEFB4FF03C4
:10678F007F00229001F5E4F09001F4E4F090009581
:10679F00E0FFEFD39406500302686990005BE0FFBF
:1067AF00EF04FF9001F2EFF09001F3E4F09001F3AA
:1067BF00E0FFEFC3941540030268629001F2E0FF1F
:1067CF00EFD3941440069001F27401F09001F2E0BF
:1067DF00FF74EE2FF582E43400F583E0FFEF64FFE2
:1067EF0070629001F2E0FF74BE2FF582E43400F581
:1067FF0083E0FF90005BE0FE74BE2EF582E4340070
:10680F00F583E0FEEEC39F403B9001F2E0FF74BEC4
:10681F002FF582E43400F583E0FF9001F4E0FEEF02
:10682F00D39E40209001F2E0FF9001F5EFF0900130
:10683F00F2E0FF74BE2FF582E43400F583E0FF90A1
:10684F0001F4EFF09001F3E004F09001F2E004F0B6
:10685F000267BC9001F5E0FF222290005BE0FFEFA2
:10686F0014FF9001F2EFF09001F3E4F09001F3E0E8
:10687F00FFEFC39415400302691E9001F2E0FFEF92
:10688F0070069001F27414F09001F2E0FF74EE2F95
:10689F00F582E43400F583E0FFEF64FF706290014E
:1068AF00F2E0FF74BE2FF582E43400F583E0FF9031
:1068BF00005BE0FE74BE2EF582E43400F583E0FE4B
:1068CF00EEC39F403B9001F2E0FF74BE2FF582E4D0
:1068DF003400F583E0FF9001F4E0FEEFD39E4020FB
:1068EF009001F2E0FF9001F5EFF09001F2E0FF74FC
:1068FF00BE2FF582E43400F583E0FF9001F4EFF052
:10690F009001F3E004F09001F2E014F002687B9044
:04691F0001F5E0FF9F
:016923002251
:109B700090005BE0FFEFD3941440037F202290001D
:049B80005BE0FF2285
:10797B00900157E0FFEFD394144006900157740128
:10798B00F09000E7E4F0900157E0FF742D2FF582A3
:10799B00E43401F583E0FF900157E0FE74032EF50C
:1079AB0082E43401F583E0FEEEB50726900157E043
:1079BB00FF74422FF582E43401F583E0FF90015709
:1079CB00E0FE74EE2EF582E43400F583E0FEEE6FFC
:1079DB0060069000E77401F0900157E0FF74EE2F02
:1079EB00F582E43400F583E0FF90005BE0FEEF6E80
:1079FB00600E90005BE0FF900157E0FEEE6F703A77
:107A0B009000E7E0FFEF6043900157E0FFEFD39466
:107A1B00155014900157E0FF74182FF582E43401D0
:107A2B00F5837401F08024900157E0FF74182FF553
:107A3B0082E43401F583E4F08011900157E0FF7488
:107A4B00182FF582E43401F583E4F09000E7E0FFB2
:107A5B00EF6044900157E0FF74032FF582E434018B
:107A6B00F583E0FF900157E0FE742D2EF582E43490
:107A7B0001F583EFF0900157E0FF74EE2FF582E4F0
:107A8B003400F583E0FF900157E0FE74422EF5823F
:0E7A9B00E43401F583EFF0900157E004F0228F
:10734200900198E0FFEF60030273F0900006E0FF07
:10735200EF70037F012212957FEFB40105127ABB11
:107362008003127AC1204A037F002212957FEF64C4
:10737200017078304A72C24A1271EB90004EE0FFFF
:10738200900194EFF090004FE0FF900195EFF090A4
:10739200004DE0FF900196EFF0900196E0FFEFB410
:1073A2001F14900192E0FF900195E0FEEEB50706F2
:1073B200127AC17F0122900191E0FF900194E0FED8
:1073C200EEB5070E900192E0FF900195E0FEEE6FA0
:1073D20060099001987401F07F002290008CE0FF18
:1073E200900006EFF07F00227F00227F00229001B2
:1073F20098E0FFEF6401600302748E900006E0FFE4
:10740200EF70037F012212957FEFB40105127ABB60
:107412008003127AC1204A037F0022C24A1271EB12
:1074220090004EE0FF900194EFF090004FE0FF904B
:107432000195EFF090004DE0FF900196EFF0900182
:1074420096E0FFEFB41F14900192E0FF900195E0E7
:10745200FEEEB50706127AC17F0122900191E0FF8C
:10746200900194E0FEEEB50720900192E0FF9001BA
:1074720095E0FEEEB5071290008CE0FF900006EF5B
:10748200F0900198E4F07F00227F0022900198E4BE
:04749200F07F002265
:10957F00900083E0FFEF600D127AE540047F0180D9
:10958F00027F002222900084E0FFEF60139000859D
:10959F00E0FFE532D39F40047F0122227F00222289
:1095AF00900085E0FFE532C39F50047F0122227FA8
:0295BF00002288
:10708F0090019DE0FFEF6003027141900008E0FF67
:10709F00EF70037F012212957FEFB40105127ABBC7
:1070AF008003127AC190019CE0FFEFB40106203BF0
:1070BF00037F002290019CE0FFEFB4020620410302
:1070CF007F002212957FEF6401706490019CE0FFB6
:1070DF00EF64017021303B1EC23BE53F653E600906
:1070EF0090019D7401F07F0022900091E0FF9000CD
:1070FF0008EFF07F002290019CE0FFEF6402702FF9
:10710F0030412CC24190019FE534F090019FE0FF88
:10711F0090019EE0FEEE6F600990019D7401F07F7B
:10712F000022900091E0FF900008EFF07F00227F97
:10713F00002290019DE0FFEF640160030271EA906D
:10714F000008E0FFEF70037F012212957FEFB4017B
:10715F0005127ABB8003127AC190019CE0FFEFB455
:10716F000106203B037F002290019CE0FFEFB40259
:10717F00062041037F002212957FEF6401705A9021
:10718F00019CE0FFEFB4011C303B19C23BE53FB55A
:10719F003E1290019DE4F0900091E0FF900008EF07
:1071AF00F07F002290019CE0FFEF6402702B3041D2
:1071BF0028C24190019FE534F090019FE0FF9001BC
:1071CF009EE0FEEEB5071290019DE4F0900091E075
:0C71DF00FF900008EFF07F00227F0022EC
:108F54007BFF7A6A79C4129845127AE5400B7BFF4D
:108F64007A6A79D512987A80097BFF7A6A79E6124F
:108F7400987A7F17127ED6AF32127B8C900054E021
:108F8400FF127EA7900055E0FF127EA7900056E0E6
:108F9400FF127EA77F1C127ED6AF31127B8C90000D
:108FA40054E0FF127EA7900055E0FF127EA79000C8
:078FB40056E0FF127EA72228
:10997500900088E0FFEF6013900089E0FFE531D3A8
:109985009F40047F0122227F002222900089E0FF70
:0D999500E531C39F50047F0122227F002294
:109BEC00900083E0FFEF6004128C1E22126DC922DC
:108C1E009001A5E0FFEF7016127AE5407290008683
:108C2E00E0FF90000AEFF09001A5E004F022900121
:108C3E00A5E0FFEF64017028127AE5401C90000A4F
:108C4E00E0FFEF704AD25B900090E0FF900007EFDC
:108C5E00F09001A5E004F022229001A5E4F022227A
:108C6E009001A5E0FFEFB40221127AE5400B9000CF
:108C7E0090E0FF900007EFF022900007E0FFEF700A
:108C8E000EC25B9001A5E4F022229001A5E4F02231
:106DC9009001A5E0FFEF704C900084E0FFEF602395
:106DD900900085E0FFE532D39F4013900086E0FFE5
:106DE90090000AEFF09001A5E004F0228026C25B32
:106DF900228021900085E0FFE532C39F5013900067
:106E090086E0FF90000AEFF09001A57403F022805C
:106E190003C25B229001A5E0FFEF64017035900089
:106E290085E0FFEF24FBFFE532D39F401F90000A66
:106E3900E0FFEF6003026F2CD25B900087E0FF90C8
:106E4900000BEFF09001A5E004F022229001A5E4E7
:106E5900F022229001A5E0FFEF6402702E900085D8
:106E6900E0FFEF24FBFFE532D39F400B900087E062
:106E7900FF90000BEFF02290000BE0FFEF600302A0
:106E89006F2CC25B9001A5E4F022229001A5E0FFDE
:106E9900EF64037043900085E0FF7E00EF2405FF57
:106EA900EE3400FEAD327C00C3ED9FEE6480F8EC59
:106EB900648098501C90000AE0FFEF7066D25B90E6
:106EC9000087E0FF90000BEFF09001A5E004F022AD
:106ED900229001A5E4F022229001A5E0FFEF6404CD
:106EE900703C900085E0FF7E00EF2405FFEE340042
:106EF900FEAD327C00C3ED9FEE6480F8EC648098AF
:106F0900500B900087E0FF90000BEFF02290000BF0
:106F1900E0FFEF700EC25B9001A5E4F02222900120
:046F2900A5E4F022C9
:109B2D0012676F8F1D9001E6E0FFEF651D600890D5
:079B3D0001E6E51DF0D25C1A
:019B440022FE
:107CF30090005BE0FFEF12866D7D3C017D46027DC7
:107D030050037D5A047D64057D6E067D78077D8270
:107D1300087D8C097D960A7DA00B7DAA0C7DB40D90
:107D23007DBE0E7DC80F7DD2107DDC117DE6127DF8
:107D3300F0137DFA1400007E037BFF7A6A79F71251
:107D4300987A227BFF7A6B790812987A227BFF7AE2
:107D53006B791912987A227BFF7A6B792A12987AB7
:107D6300227BFF7A6B793B12987A227BFF7A6B79BD
:107D73004C12987A227BFF7A6B795D12987A227B78
:107D8300FF7A6B796E12987A227BFF7A6B797F1276
:107D9300987A227BFF7A6B799012987A227BFF7A0A
:107DA3006B79A112987A227BFF7A6B79B212987A57
:107DB300227BFF7A6B79C312987A227BFF7A6B79E5
:107DC300D412987A227BFF7A6B79E512987A227B18
:107DD300FF7A6B79F612987A227BFF7A6C79071215
:107DE300987A227BFF7A6C791812987A227BFF7A31
:107DF3006C792912987A227BFF7A6C793A12987AF5
:017E0300225C
:105601002020464C45582049562030303720202054
:10561100002049502050524F4752414D4D494E476D
:10562100200043544353532036332E302020202072
:10563100202043544353532036372E30202020203E
:10564100202043544353532036392E342020202028
:10565100202043544353532037312E39202020201A
:10566100202043544353532037342E34202020200C
:10567100202043544353532037372E3020202020FD
:10568100202043544353532037392E3720202020E4
:10569100202043544353532038322E3520202020DC
:1056A100202043544353532038352E3420202020CA
:1056B100202043544353532038382E3520202020B6
:1056C100202043544353532039312E3520202020AC
:1056D100202043544353532039342E382020202096
:1056E100202043544353532039372E342020202087
:1056F10020204354435353203130302E302020207A
:1057010020204354435353203130332E3520202061
:1057110020204354435353203130372E3220202050
:1057210020204354435353203131302E392020203F
:1057310020204354435353203131342E382020202C
:1057410020204354435353203131382E3820202018
:1057510020204354435353203132332E3020202014
:1057610020204354435353203132372E33202020FD
:1057710020204354435353203133312E38202020ED
:1057810020204354435353203133362E35202020DB
:1057910020204354435353203134312E33202020D1
:1057A10020204354435353203134362E32202020BD
:1057B10020204354435353203135312E34202020AF
:1057C10020204354435353203135362E3720202097
:1057D10020204354435353203135392E3820202083
:1057E10020204354435353203136322E322020207F
:1057F10020204354435353203136352E3520202069
:1058010020204354435353203136372E3920202052
:1058110020204354435353203137312E332020204D
:1058210020204354435353203137332E3820202036
:1058310020204354435353203137372E3320202027
:1058410020204354435353203137392E392020200F
:1058510020204354435353203138332E3520202008
:1058610020204354435353203138362E32202020F8
:1058710020204354435353203138392E39202020DE
:1058810020204354435353203139322E38202020D5
:1058910020204354435353203139362E36202020C3
:1058A10020204354435353203139392E35202020B1
:1058B10020204354435353203230332E35202020AF
:1058C10020204354435353203230362E352020209C
:1058D10020204354435353203231302E372020208F
:1058E10020204354435353203231382E312020207D
:1058F10020204354435353203232352E3720202069
:1059010020204354435353203232392E312020205A
:1059110020204354435353203233332E362020204A
:1059210020204354435353203234312E3820202039
:1059310020204354435353203235302E332020202E
:1059410020204354435353203235342E312020201C
:105951002020202020202020202020202020202046
:02596100202004
:1062470075840F1265BA9001E87401F09001E97442
:1062570003F07D007CFC7F1012963FE49001E8F08C
:106267009001E9F020A10875840F43E8C080067506
:10627700840F53E83F129BFC7BFF7A5679011298F3
:1062870045129B45900003741EF0900003E070FADE
:10629700129BA990005BE0FF6005D3941440069021
:1062A700005B7401F0127CF31288591290E412918A
:1062B700401298AF127AAF900099E0FF789F76006E
:1062C70008A6079000A4E09001A6F0E49000EDF086
:1062D700900190F090018FF0900198F09001A0F05C
:1062E70090005274FFF0900053F0E49001E6F090B4
:1062F70001E5F0F558127AC1304313124A90129B08
:10630700A91288591290E4129140C24380EA20A64C
:106317000E128F54E4900190F090018FF080EF30CF
:10632700461DC246124A90129BA91288591290E440
:10633700129140129BFCE490018FF0900190F04382
:10634700E7403058061290211299FA30A704C2A7E5
:106357008002D2A71241EE12328612770FE55BB4A4
:106367005514E55CB4AA0F9001E77414F09001E7A7
:10637700E070FA127AB59001A7E07040127AC75020
:106387003B127BD512797B125A47129BEC129084F1
:10639700129B2D305C1E205D1BC25C9001E6E02441
:1063A70000FEE434179001C2F0A3CEF09001BE7452
:1063B70001F0D25DE49001F9F0026315127AAF9013
:1063C7000099E0FF789F760008A6079000A4E09068
:1063D70001A6F0E4900190F090018FF0900198F001
:1063E70090005BE0900052F090005374FCF0127A3A
:0D63F700C17BFF7A567912126C4B026315C0
:108FBB0001AE01C901DA01EB01FC020E0220023302
:108FCB000247025C02710287029902AB02C302DC08
:108FDB0002F50310032B03480365038403A403C5A5
:108FEB0003E6040A042E04430453046A047A04912E
:108FFB0004A204BA04CC04E504F705100524053ECD
:10900B000552056D0582059E05D10605061C063B1E
:06901B00067306AD06C756
:109AC200C23DC23FEF25E024BBF582E4348FF5832B
:0E9AD200E493F51A740193F51BD23ED23822AC
:09009600C23DC23FC23EC2382245
:0300A30002953C87
:10953C00C0E0C0F0C083C082C0D075D000C000C0F5
:10954C0001C002C003C004C005C006C007205805F6
:10955C00128206800312924BD007D006D005D0049D
:10956C00D003D002D001D000D0D0D082D083D0F0A4
:03957C00D0E0320A
:03009300028E17C3
:0B8E1700C0E0C0D075D000C006C0074E
:108E2200AE84758402E5337007AFBE75BB07802F31
:108E3200E533B40107AFBE75BB048023E533B4024A
:108E420007AFBE75BB068017E533B4030885BE3194
:108E520075BB04800AE533B40409AFBE75BB0505D2
:108E6200338010E533B4050885BE3275BB0480003B
:078E7200753300C2ED8E8490
:098E7900D007D006D0D0D0E032C1
:03008300029602E0
:10960200C0E0C0F0C083C082C0D075D000C000C02E
:1096120001C002C003C004C005C006C007C2CF1209
:109622001CD0D007D006D005D004D003D002D00180
:0D963200D000D0D0D082D083D0F0D0E03274
:0300730002897D82
:10897D00C0E0C0F0C083C082C0D075D000C000C0C0
:10898D0001C002C003C004C005C006C007C2CF307D
:10899D005805128EEC80031291F57895E66001165C
:1089AD00304027C240D54A05754A0A05491275D38C
:1089BD00D51C09751C0A758401438820D5301B759B
:1089CD0030607584024388208010D2401278F1788F
:1089DD009616E670057604121A1A758401438810EE
:1089ED00758402D2ECD007D006D005D004D003D0C8
:1089FD0002D001D000D0D0D082D083D0F0D0E032E0
:03006B000293E518
:1093E500C0E0C0F0C083C082C0D075D000C000C04E
:0D93F50001C002C003C004C005C006C007CF
:0E9402008584721282DA758402C28D857284AE
:10941000D007D006D005D004D003D002D001D000B0
:0B942000D0D0D082D083D0F0D0E0325A
:03005B0002939776
:10939700C0E0C0F0C083C082C0D075D000C000C09C
:1093A70001C002C003C004C005C006C00712597C33
:1093B7007897E6600116900007E0600214F0758464
:1093C70001C28DD007D006D005D004D003D002D07B
:0E93D70001D000D0D0D082D083D0F0D0E032D0
:0300530002942BE9
:10942B00C0E0C0F0C083C082C0D075D000C000C007
:10943B0001C002C003C004C005C006C007C28C3007
:10944B005904C2598005D2591275F5D007D006D0F0
:10945B0005D004D003D002D001D000D0D0D082D020
:06946B0083D0F0D0E032D6
:03002B00020016BA
:03001600C2CF3224
:03002300029B97A6
:109B9700309904C299C262309807859956C298D203
:029BA700613229
:03001B00020019C7
:0100190032B4
:10947100A984A2AF9264AEB1C2AF75840F53A1FEAD
:109481008FB1E4F5849001E8E042B79001E9E04250
:109491008F8C088D098D828C83EBF0E4F58490012B
:1094A100E9E0F4528F9001E8E0F452B78EB189847B
:0494B100A26492AF70
:0194B5002294
:10963F00A984A2AF9264AEB1C2AF8C088D098FB16D
:10964F00E4F5849001E8E0FF42B7E4F5849001E986
:10965F00E0FD428F850982850883E4F0EDF4528F97
:0C966F00EFF452B78EB18984A26492AF70
:01967B0022CC
:109A6300AE84A2AF9264ABB1C2AF8FB18C0A8D0B3F
:0F9A73008D828C83E493FF8BB18E84A26492AFBB
:019A820022C1
:100EC800202020464C45582049562020202020200C
:100ED8000020202020202020202020202049444CB1
:100EE80045002054657374696E67204D6F646520F2
:100EF80020200043726F73732042757379204D6F01
:100F08006465200053656E642049646C654D6573A3
:100F1800736167650043726F73732042757379203C
:100F28004D6F6465310043726F7373204275737936
:100F3800204D6F6465320043726F7373204275737E
:100F480079204D6F6465330043726F737320427567
:100F58007379204D6F64653400202053656E646991
:100F68006E672043574944202000205741495420A8
:100F78005544544420464C414720004C5452564F47
:100F88004950204F5554474F494E470020564F4926
:100F980050204F5554474F494E47202000202049A4
:100FA8004E434F4D494E47204C545220200020209C
:100FB800494E434F4D494E472043544353532020F5
:100FC800002020494E434F4D494E4720444353206B
:100FD800200043544353532036332E302020202002
:100FE800202043544353532036372E3020202020CE
:100FF800202043544353532036392E3420202020B8
:10100800202043544353532037312E3920202020A9
:10101800202043544353532037342E34202020209B
:10102800202043544353532037372E30202020208C
:10103800202043544353532037392E372020202073
:10104800202043544353532038322E35202020206B
:10105800202043544353532038352E342020202059
:10106800202043544353532038382E352020202045
:10107800202043544353532039312E35202020203B
:10108800202043544353532039342E382020202025
:10109800202043544353532039372E342020202016
:1010A80020204354435353203130302E3020202009
:1010B80020204354435353203130332E35202020F1
:1010C80020204354435353203130372E32202020E0
:1010D80020204354435353203131302E39202020CF
:1010E80020204354435353203131342E38202020BC
:1010F80020204354435353203131382E38202020A8
:1011080020204354435353203132332E30202020A3
:1011180020204354435353203132372E332020208C
:1011280020204354435353203133312E382020207C
:1011380020204354435353203133362E352020206A
:1011480020204354435353203134312E3320202060
:1011580020204354435353203134362E322020204C
:1011680020204354435353203135312E342020203E
:1011780020204354435353203135362E3720202026
:1011880020204354435353203135392E3820202012
:1011980020204354435353203136322E322020200E
:1011A80020204354435353203136352E35202020F8
:1011B80020204354435353203136372E39202020E2
:1011C80020204354435353203137312E33202020DD
:1011D80020204354435353203137332E38202020C6
:1011E80020204354435353203137372E33202020B7
:1011F80020204354435353203137392E392020209F
:1012080020204354435353203138332E3520202097
:1012180020204354435353203138362E3220202087
:1012280020204354435353203138392E392020206D
:1012380020204354435353203139322E3820202064
:1012480020204354435353203139362E3620202052
:1012580020204354435353203139392E3520202040
:1012680020204354435353203230332E352020203E
:1012780020204354435353203230362E352020202B
:1012880020204354435353203231302E372020201E
:1012980020204354435353203231382E312020200C
:1012A80020204354435353203232352E37202020F8
:1012B80020204354435353203232392E31202020EA
:1012C80020204354435353203233332E36202020DA
:1012D80020204354435353203234312E38202020C9
:1012E80020204354435353203235302E33202020BE
:1012F80020204354435353203235342E31202020AC
:1013080020202020202020202020202020202020D5
:1013180020204443532030303620494E5620303266
:1013280031204443532030303720494E5620323143
:1013380034204443532030313520494E562031342F
:1013480031204443532030313720494E5620303520
:1013580030204443532030323120494E562030301B
:1013680036204443532030323320494E56203034FF
:1013780037204443532030323520494E56203234EA
:1013880034204443532030323620494E56203436D8
:1013980034204443532030333120494E56203632CE
:1013A80037204443532030333220494E56203035BD
:1013B80031204443532030333620494E56203137AC
:1013C80032204443532030343320494E562034349D
:1013D80035204443532030343720494E562030328C
:1013E80033204443532030353020494E5620303185
:1013F80037204443532030353120494E562030336E
:1014080032204443532030353320494E562034355A
:1014180032204443532030353420494E562034314D
:1014280033204443532030363520494E5620323736
:1014380031204443532030373120494E5620333031
:1014480036204443532030373220494E5620323418
:1014580035204443532030373320494E5620353009
:1014680036204443532030373420494E56203137F4
:1014780034204443532031313420494E56203731EB
:1014880032204443532031313520494E56203135DE
:1014980032204443532031313620494E56203735C7
:1014A80034204443532031323220494E56203232C0
:1014B80035204443532031323520494E56203336A7
:1014C80035204443532031333120494E562033369A
:1014D80034204443532031333220494E562035348A
:1014E80036204443532031333420494E562032327B
:1014F80033204443532031343120494E5620303173
:1015080035204443532031343320494E562034315A
:1015180032204443532031343520494E5620323747
:1015280034204443532031353220494E562031313E
:1015380035204443532031353520494E5620373322
:1015480031204443532031353620494E5620323617
:1015580035204443532031363220494E5620353009
:1015680033204443532031363520494E56203235F6
:1015780031204443532031373220494E56203033EE
:1015880036204443532031373420494E56203037D3
:1015980034204443532032303520494E56203236C9
:1015A80033204443532032313220494E56203335BC
:1015B80036204443532032313420494E56203030AF
:1015C80037204443532032323320494E562031339A
:1015D80034204443532032323520494E562031328C
:1015E80032204443532032323620494E562034317B
:1015F80031204443532032343320494E562033356A
:1016080031204443532032343420494E562030325E
:1016180035204443532032343520494E5620303744
:1016280032204443532032343620494E5620353236
:1016380033204443532032353120494E5620313629
:1016480035204443532032353220494E5620343613
:1016580032204443532032353520494E5620343405
:1016680036204443532032363120494E56203733F2
:1016780032204443532032363320494E56203230EC
:1016880035204443532032363520494E56203135D3
:1016980036204443532032363620494E56203435BE
:1016A80034204443532032373120494E56203036B7
:1016B80035204443532032373420494E56203134A4
:1016C80035204443532033303620494E5620303796
:1016D80031204443532033313120494E5620363689
:1016E80034204443532033313520494E5620343278
:1016F80033204443532033323520494E5620353267
:1017080036204443532033333120494E5620343653
:1017180035204443532033333220494E5620343544
:1017280035204443532033343320494E5620353333
:1017380032204443532033343620494E5620363124
:1017480032204443532033353120494E5620323419
:1017580033204443532033353620494E5620323106
:1017680032204443532033363420494E56203133F7
:1017780031204443532033363520494E56203132E8
:1017880035204443532033373120494E56203733D0
:1017980034204443532034313120494E56203232CC
:1017A80036204443532034313220494E56203134B8
:1017B80033204443532034313320494E56203035AA
:1017C80034204443532034323320494E5620333199
:1017D80035204443532034333120494E5620373284
:1017E80033204443532034333220494E5620353178
:1017F80036204443532034343520494E5620303463
:1018080033204443532034343620494E5620323551
:1018180035204443532034353220494E5620303544
:1018280033204443532034353420494E5620323631
:1018380036204443532034353520494E562033331F
:1018480032204443532034363220494E5620323514
:1018580032204443532034363420494E5620303207
:1018680036204443532034363520494E56203333EE
:1018780031204443532034363620494E56203636DC
:1018880032204443532035303320494E56203136D8
:1018980032204443532035303620494E56203037C5
:1018A80033204443532035313620494E56203433B3
:1018B80032204443532035323320494E56203234A7
:1018C80036204443532035323620494E5620333291
:1018D80035204443532035333220494E5620333483
:1018E80033204443532035343620494E5620313373
:1018F80032204443532035363520494E5620373060
:1019080033204443532036303620494E5620363350
:1019180031204443532036313220494E5620333447
:1019280036204443532036323420494E562036332D
:1019380032204443532036323720494E5620303324
:1019480031204443532036333120494E5620363017
:1019580036204443532036333220494E56203632FF
:1019680034204443532036353420494E56203734EA
:1019780033204443532036363220494E56203436DD
:1019880036204443532036363420494E56203331CE
:1019980031204443532037303320494E56203536C2
:1019A80035204443532037313220494E56203131B7
:1019B80034204443532037323320494E56203433A1
:1019C80031204443532037333120494E5620313596
:1019D80035204443532037333220494E562032367F
:1019E80031204443532037333420494E562033376F
:1019F80031204443532037343320494E562036355E
:101A080034204443532037353420494E5620313151
:021A1800362076
:107BD5009000B3E0FFB4010A90005274FFF0E40294
:107BE5007CA2EF64026003027CA7127AA9787BE687
:107BF5006003027C96305703027C96900197E070F3
:107C050032D23F90009AE024FF924D90005BE0FF56
:107C150090015BF0900098E090015CF090015DEFC1
:107C2500F012692490015EEFF0128693900197742B
:107C350002F0221283AEEF64017050D23F900158DA
:107C4500E0FF2442F582E43401F583E090015BF026
:107C5500742D2FF582E43401F583E090015CF090FA
:107C65000158E090015DF012640490015EEFF09020
:107C7500015BE024D2F582E43400F583E024FF9231
:107C85004D128693900197E014F022900197E0142D
:107C9500F090005BE0900052F0900098E090005367
:107CA500F02290018FE0B40900503D907CB7F82890
:107CB5002873027CD2027CD5027CD8027CDB027C54
:107CC500DE027CE1027CE4027CE7027CEA0224D548
:107CD500028A940288EC025294024653022D06024F
:0E7CE5003CFB024EA10237EEE490018FF0222C
:1024D500900190E0B40C004003022D009024E8F830
:1024E50028287302250C0225400227D70228150249
:1024F50028380228620229280229B2022A44022A1F
:1025050071022B36022C0BE49001E5F07BFF7A0E6D
:1025150079C81298457BFF7A0E79D912987A90007E
:102525005274FFF0900053F0127AAF9000B4E0605F
:1025350003127AD39001907401F02220A55C127ADF
:10254500A99000B4E06003127ACD9000B1E090004C
:1025550000F090005BE0FF900052F0900098E0FEE4
:10256500900053F09001907405F090015BEFF090AE
:10257500015CEEF090005BE090015DF01264049068
:10258500015EEFF090009AE024FF924D128693D2FF
:102595003F7BFF7A0E79EA0298459001E2E06403F9
:1025A5007034127AA99000B4E06003127ACD9000DD
:1025B500B1E0900000F0E49001E2F09001E3E090DA
:1025C5000052F09001E4E0900053F0E4900190F0A7
:1025D50090018F0229A09001E2E0602D127AA99066
:1025E50000B4E06003127ACD9000B1E0900000F0F5
:1025F50090005BE0900052F090005374FEF0E49080
:102605000190F090018F022A40305B61304A5EC232
:102615004A90004EE0FFC39415505274D22FF582B4
:10262500E43400F583E0FFA248E4336F703FA2482D
:10263500924990004EE0900191F090004FE090019A
:1026450092F090004DE0900193F01271EB900193A0
:10265500E0641F6018900191E0FF900192E0FD7C1D
:102665000012872E90018F7402F0022D00C24A12CB
:10267500002EBF0117127AA99000B4E06003127A08
:10268500CD9000B1E0900000F0022A2E9000B5E058
:10269500602512957FEF64016006129975BF0117D9
:1026A5007BFF7A0E79FB129845900092E0789EF6B2
:1026B5009001907409F02212957FEF6401706830E3
:1026C5003B28C23B90019C04F0D239853E3FE53F53
:1026D50075F010A424DAF9740F35F0FA7BFF12981F
:1026E50045AF3F128D1DC239802A30413AC2419013
:1026F500019EE534F075F010A4241AF9741335F031
:10270500FA7BFF12984590019EE0FF128B1A90010B
:102715009C7402F090018F7405F0E4900190F090A4
:102725000092E0789EF622C23BC24178A0E61846A8
:10273500703F900099E060397BFF7A0F790C129811
:1027450045900099E0FF789F760008A60790005213
:1027550074FFF0900053F0127AA99000B4E0600382
:10276500127ACD9000B1E0900000F0900190022C1B
:102775008F9000A4E0FF7003022D059001A6E06094
:1027850003022D059000A2E0FE60107003022D05E6
:102795009001A2E064016003022D059001A6EFF00F
:1027A500E49001A2F0127AA99000B4E06003127AD5
:1027B500CD9000B1E0900000F090005BE0900052F9
:1027C500F090005374FDF0E4900190F090018F04B7
:1027D500F022900000E06003022D05305703022D22
:1027E5000590005BE0FF90015BF090015C74FFF0E9
:1027F50090015DEFF090015EF090009AE024FF9269
:102805004D128693D23F12728D9001907403F0227F
:10281500787BE66003022D05305703022D05127EF5
:10282500F0127EFF90008DE0900001F09001907411
:1028350004F022900001E06003022D05127AAF90AA
:1028450000B4E06003127AD3E4900190F09001A205
:1028550004F090005274FFF0900053F02230A5036D
:1028650002292590005BE0900052F0900098E090DE
:102875000053F012957FBF0105127ABB8003127ACF
:10288500C1787BE66003022D05305703022D0590C4
:102895000197E07034D23F90009AE024FF924D906A
:1028A500005BE0FF90015BF0900098E090015CF028
:1028B50090015DEFF012692490015EEFF0128693AE
:1028C5009001977402F002728D1283AEEF6401706D
:1028D5004CD23F900158E0FF2442F582E43401F5E3
:1028E50083E090015BF0742D2FF582E43401F583CC
:1028F500E090015CF0900158E090015DF0126404F5
:1029050090015EEFF090015BE024D2F582E43400A3
:10291500F583E024FF924D128693022CE4022CE409
:10292500022D00900000E06003022D0530570302E0
:102935002D05787BE66003022D0590005274FFF0AB
:10294500900053F012847CEF64017053900158E0BD
:10295500FF2442F582E43401F583E090015BF074D5
:102965002D2FF582E43401F583E090015CF09001B0
:1029750058E090015DF0129B7090015EEFF09001C0
:102985005BE024D2F582E43400F583E024FF924D28
:10299500128693D23F12728D9001907407F02290A7
:1029A500008DE0900001F0900190022A40305B63B9
:1029B500304A62C24A90004EE0FFC39415505674E7
:1029C500D22FF582E43400F583E0FFA248E4336FAB
:1029D5007043A248924990004EE0900191F090001A
:1029E5004FE0900192F090004DE0900193F012714C
:1029F500EB900193E0641F601C900191E0FF900152
:102A050092E0FD7C0012872EE4900190F090018FFA
:102A1500022C8FC24A787BE66003022D05305703EE
:102A2500022D0512002EEF60079001907406F0222A
:102A350090008DE0900001F09001907408F02290D4
:102A45000001E06003022D05127AAF9000B4E0604A
:102A550003127AD39001A27401F0E4900190F090F2
:102A6500005274FFF0900053F0027EFF305B63303C
:102A75004A60C24A90004EE0FFC39415505474D288
:102A85002FF582E43400F583E0FFA248E4336F704C
:102A950041A248924990004EE0900191F090004F7C
:102AA500E0900192F090004DE0900193F01271EBEF
:102AB500900193E0641F601A900191E0FF900192EC
:102AC500E0FD7C0012872EE4900190F090018F02CA
:102AD5002C8FC24A789EE66003022D0590005BE0CC
:102AE500900052F090005374FDF09000B5E0FF6443
:102AF500016004EFB4021512957FBF010F9000939A
:102B0500E0900005F0900190740AF0229000B5E085
:102B1500FF64036004EFB40415129975BF010F90AB
:102B25000093E0900005F0900190740BF022022DC7
:102B35000012957FBF0108900093E0900005F0908A
:102B45000005E07003022C1F9000B5E0B401097B7D
:102B5500FF7A0F791D022C3E127AA97BFF7A0F7935
:102B65002E12987A787BE66003022CF13057030227
:102B75002CF1900197E07031D23F90009AE024FF4C
:102B8500924D90005BE0FF90015BF0900098E09023
:102B9500015CF090015DEFF012692490015EEFF0A9
:102BA500128693900197022C8F1283AEEF64017009
:102BB5004CD23F900158E0FF2442F582E43401F500
:102BC50083E090015BF0742D2FF582E43401F583E9
:102BD500E090015CF0900158E090015DF012640412
:102BE50090015EEFF090015BE024D2F582E43400C1
:102BF500F583E024FF924D128693022CE490019711
:102C0500E014F0022CF1129975BF0108900093E0D1
:102C1500900005F0900005E07012127AAF900099CF
:102C2500E0FF789F760008A607022D009000B5E02A
:102C3500B403097BFF7A0F793F02987A7BFF7A0FFD
:102C4500795012987A127AA9787BE66003022CF102
:102C5500305703022CF1900197E07032D23F90007B
:102C65009AE024FF924D90005BE0FF90015BF090AD
:102C75000098E090015CF090015DEFF012692490FE
:102C8500015EEFF01286939001977402F022128391
:102C9500AEEF64017050D23F900158E0FF2442F539
:102CA50082E43401F583E090015BF0742D2FF58209
:102CB500E43401F583E090015CF0900158E0900167
:102CC5005DF012640490015EEFF090015BE024D2A8
:102CD500F582E43400F583E024FF924D128693904B
:102CE5000197E014F022900197E014F090005BE06A
:102CF500900052F090005374FDF022E4900190F0A2
:012D050022AB
:108A940012919C900190E0FF700C900000E07075C2
:108AA40090019004F022EF64017029205D1D900173
:108AB400C27419F0A3E4F09001BE04F0D25D9001F9
:108AC4009004F07BFF7A0F796180067BFF7A0F793F
:108AD4007202987A900190E0FFB402189001E5E0E8
:108AE40064017031F090008DE0900001F0900190ED
:108AF4007403F022EFB40314900001E07017127AAB
:108B0400AF9000B4E06005127AD38000E490018F46
:068B1400F0900190F02238
:1088EC00900190E0703B900068E0602B127AA990A8
:1088FC0000B4E06003127ACD9000B1E0900000F07B
:10890C00900191E0900052F0900192E0900053F0B1
:10891C009001907401F022E4900190F090018FF09E
:10892C0022900190E06401703E205D32900191E054
:10893C00FE900192E07C002400FFEC3E9001C2F01E
:10894C00A3EFF09001BE7401F0D25D900069E0904D
:10895C00018F6004740480027403F0E4800E7BFFCA
:10896C007A0F797202987AE490018FF0900190F06E
:01897C0022D8
:10529400900190E0704A900000E06003025600A282
:1052A40049924D900191E090015BF0900192E09061
:1052B400015CF090005BE090015DF01269249001C4
:1052C4005EEFF0128693D23F12728D9001977408AC
:1052D400F090008CE0900006F09001907401F022B0
:1052E400900190E06401703E127342EF60028055B9
:1052F400787BE66003025600305703025600762896
:10530400D257900197E014F0E06003025600740253
:10531400F090008CE0900006F090008EE090000C7D
:10532400F09001908069900190E064026003025360
:10533400F1127342EF6002800C90008EE0600D90D9
:10534400000CE070079001907403F022787BE66013
:1053540003025600305703025600900197E0703361
:10536400A249924D900191E090015BF0900192E08E
:1053740090015CF090005BE090015DF01269249074
:10538400015EEFF0128693D23F12728D90019774F2
:1053940002F0221283AEEF6401704F900158E0FFD7
:1053A4002442F582E43401F583E090015BF0742D2E
:1053B4002FF582E43401F583E090015CF09001580C
:1053C400E090015DF012640490015EEFF090015BE7
:1053D400E024D2F582E43400F583E024FF924D12F8
:1053E4008693D23F12728D0254A40254A490019069
:1053F400E06403702E205D229001C2F0A374FFF0DC
:105404009001BE7401F0D25D127EF0127AC1E49074
:105414000198F09001907404F0227BFF7A0F797266
:1054240002987A900190E064047043787BE660030C
:10543400025600305703025600A249924D90019142
:10544400E090015BF0900192E090015CF090015DCE
:10545400741FF0129B7090015EEFF012869390011E
:10546400977403F012728D9001907405F0229001EC
:1054740090E0FF64057030787BE6600302560030EC
:105484005703025600900197E0700F90008DE09052
:105494000001F09001907406F022787B7628D257B0
:1054A400900197E014F022EF640660030255E9903E
:1054B40000B5E0601F303B09304106129975EF706A
:1054C40013E490018FF0900190F0900092E0789EA8
:1054D400F60255DC305B7A304A77C24A90004EE0DF
:1054E400FFC39415506B74D22FF582E43400F58316
:1054F400E0FFA248E4336F7058A248924990004EEE
:10550400E0900191F090004FE0900192F090004DF6
:10551400E0900193F0641F6038900191E0FFC39420
:1055240015502E74D22FF582E43400F583E0FFA2E7
:1055340049E433B5071B900191E0FF900192E0FD2F
:105544007C0012872E90018F7402F0E4900190F099
:1055540022C24A787BE6705520575212847CEF644D
:1055640001704A900158E0FF2442F582E43401F5C9
:1055740083E090015BF0742D2FF582E43401F58310
:10558400E090015CF0900158E090015DF012640439
:1055940090015EEFF090015BE024D2F582E43400E8
:1055A400F583E024FF924D12869312728D900001D0
:1055B400E07049127AAF9000B4E06003127AD3909D
:1055C400005274FFF0900053F09001A27401F0E4D3
:1055D40090018FF0900190F0900099E0FF789F7611
:1055E4000008A60722900190E0D39406400EE490B0
:0D55F400018FF0900190F0789FF608F622EC
:10465300900190E070107BFF7A0F79831298459058
:1046630001907401F022900190E064017059900070
:1046730000E06003024A8FA249924D900191E090BD
:10468300015BF0900192E090015CF090005BE090A0
:10469300015DF012692490015EEFF0128693D23F20
:1046A30012728D90008CE0900006F090008EE090E6
:1046B300000CF09000B8E09001A3F090019774070C
:1046C300F09001900247A6900190E06402703212CC
:1046D3009BEC787BE66003024A8F305703024A8FD4
:1046E3007628D257900197E014F0E06003024A8FD6
:1046F300127ABB9001977402F090019004F0C24AC1
:1047030022900190E064036003024804129BEC20B2
:104713005B089000B8E07002803F9000B8E0FF6053
:10472300089001A3E070028030305B0D304A0A909C
:1047330001A3EFF0C24A127ABB12957FEF70031206
:104743007AC19001E5E0B40104E402482990008EA7
:10475300E0600D90000CE070079001907404F0226B
:10476300787BE66003024A8F305703024A8F900139
:1047730097E07033A249924D900191E090015BF074
:10478300900192E090015CF090005BE090015DF09D
:1047930012692490015EEFF0128693D23F12728D5C
:1047A3009001977402F0221283AEEF6401704F9070
:1047B3000158E0FF2442F582E43401F583E09001DF
:1047C3005BF0742D2FF582E43401F583E090015CF6
:1047D300F0900158E090015DF012640490015EEFE7
:1047E300F090015BE024D2F582E43400F583E02409
:1047F300FF924D128693D23F12728D0248BA02483D
:10480300BA900190E06404702E205D229001C2F002
:10481300A374FFF09001BE7401F0D25D127EF0121A
:104823007AC1E4900198F09001907405F0227BFF27
:104833007A0F797202987A900190E0640570467855
:104843007BE66003024A8F305703024A8FA24992E4
:104853004D900191E090015BF0900192E090015C3A
:10486300F090015D741FF0129B7090015EEFF012E7
:104873008693127AC19001977403F012728D90019E
:10488300907406F022900190E0FF64067030787B0C
:10489300E66003024A8F305703024A8F900197E084
:1048A300700F90008DE0900001F09001907407F07C
:1048B30022787B7628D257900197E014F022EF6498
:1048C300076003024A789000B5E0601F303B09306F
:1048D3004106129975EF7013E490018FF0900190E7
:1048E300F0900092E0789EF6024A6B12957FEF6497
:1048F3000160030249D590008DE0900001F0204A49
:10490300030249D5C24A12957FEF6401600302494D
:10491300D5900191E0FF90004EE0FEB507129000A4
:104923004FE0FF900192E0B50706E4900195F02275
:10493300EEC3941540030249D590004EE0FF24D204
:10494300F582E43400F583E0FEA248E4336E6003AD
:104953000249D5900195E0FE701BA248924990014F
:1049630094EFF090004FE0900195F090004DE090AF
:104973000196F0805D90004EE0FF6E7055A2489264
:1049830049900191EFF090004FE0900192F0900078
:104993004DE0900193F0641F6038900191E0FFC3F4
:1049A3009415502E74D22FF582E43400F583E0FF82
:1049B300A249E433B5071B900191E0FF900192E017
:1049C300FD7C0012872E90018F7402F0E490019019
:1049D300F022787BE6706020575D12847CEF6401DF
:1049E3007055900158E0FF2442F582E43401F583C9
:1049F300E090015BF0742D2FF582E43401F583E040
:104A030090015CF0900158E090015DF01264049015
:104A1300015EEFF090015BE024D2F582E43400F50F
:104A230083E024FF924D1286939001907406F0E484
:104A330090018FF012728D900001E07038127AAFFE
:104A43009000B4E06003127AD390005274FFF090A8
:104A53000053F09001A27401F0E490018FF09001F3
:104A630090F0127EF0127EFF900099E0FF789F761F
:104A73000008A60722900190E0D39407400EE4902B
:0D4A8300018FF0900190F0789FF608F62268
:102D0600900190E06003022DEC12957FEF64017054
:102D16005B304A58C24A90004EE0FFC39415504CAF
:102D260074D22FF582E43400F583E0FFA248E43341
:102D36006F7039A248924990004EE0900191F09050
:102D4600004FE0900192F090004DE0900193F01258
:102D560071EB900193E0641F6012900191E0FF9087
:102D66000192E0FD7C0012872E023150C24A789E05
:102D7600E6600302328512957FEF6401705690007B
:102D86005EE07024127AAF9000B4E06003127AD34A
:102D96009000B5E0B4010F90005BE0900052F09017
:102DA600005374FEF0228038127AA99000B4E060D5
:102DB60003127ACD127ABB9000B1E0900000F09039
:102DC600005BE0900052F090005374FEF09001908A
:102DD6007401F022127AAF9000B4E06003127AD345
:102DE600C239E4023281900190E064017061305D85
:102DF60003022F4D90019CE0FBB4010FE53F240038
:102E0600FEE434159001C2F0A3CEF0EBB4021190AB
:102E1600019EE02400FEE434169001C2F0A3CEF039
:102E26009001BE7401F0D25D90008EE090000CF02F
:102E3600900091E0900008F0900060E0600BE49054
:102E46000190F090018F022F7590019002327590DB
:102E56000190E06402707A900000E060030232851F
:102E660090019CE064017025AF3F129AC2E53F7560
:102E7600F010A424DAF9740F35F0FA7BFF129845A6
:102E8600E53F75F010A424DAF9740F803590019CA3
:102E9600E06402600302328590019EE0FF121E5834
:102EA60090019EE075F010A4241AF9741335F0FA17
:102EB6007BFF12984590019EE075F010A4241AF944
:102EC600741335F0FA7BFF12987A9001907403F030
:102ED60022900190E06403702412708FEF600280EC
:102EE6001290008EE0700302328590000CE06003C1
:102EF600023285127EF09001907404F022900190C7
:102F0600E06404704B205D3F9001C2F0A374FFF0B3
:102F16009001BE7401F0D25D127EFF127AC1E49078
:102F2600019DF090005DE0600E90009FE09000092A
:102F3600F09001900232009000A0E0900002F012A2
:102F4600009690019080287BFF7A0F797202987A1A
:102F5600900190E064056003023060900009E07023
:102F6600121200969000A0E0900002F0900190747A
:102F760006F02212957FEF6401706B120096303BCB
:102F860030C23B90019C7401F0853E3FC239E53F5B
:102F960075F010A424DAF9740F35F0FA7BFF129855
:102FA60045AF3F128D1DE4900190F090018F0232E3
:102FB60000304132C24190019EE534F075F010A414
:102FC600241AF9741335F0FA7BFF12984590019E86
:102FD600E0FF128B1A90019C7402F0E4900190F0CD
:102FE60090018F023200C23BC24112957FEF64010D
:102FF6007065304A62120096C239C24A90004EE0AD
:10300600FFC39415505174D22FF582E43400F58332
:10301600E0FFA248E4336F703EA248924990004E0A
:10302600E0900191F090004FE0900192F090004DF9
:10303600E0900193F01271EB900193E0641F60172A
:10304600900191E0FF900192E0FD7C0012872E90A6
:10305600018F74020230DDC24A22900190E06406BC
:103066006003023159900002E070079001907407E6
:10307600F02212957FEF64017062303B2BC23B90C9
:10308600019C04F0853E3FC239E53F75F010A4244B
:10309600DAF9740F35F0FA7BFF129845AF3F128DBF
:1030A6001D90018F7405802F304131C24190019EE1
:1030B600E534F075F010A4241AF9741335F0FA7B90
:1030C600FF12984590019EE0FF128B1A90019C74A6
:1030D60002F090018F7405F0E4023192C23BC241C6
:1030E60012957FEF64017068304A65120096C23906
:1030F600C24A90004EE0FFC39415505474D22FF587
:1031060082E43400F583E0FFA248E4336F7041A205
:1031160048924990004EE0900191F090004FE09067
:103126000192F090004DE0900193F01271EB900146
:1031360093E0641F601A900191E0FF900192E0FD18
:103146007C0012872EE4900190F090018F02327578
:10315600C24A22900190E06407600302327C90002C
:1031660001E0702D127AAF9000B4E06003127AD3BA
:10317600127EFF900099E0FF789F760008A60790E0
:1031860001A27401F0C239E490018FF0900190F031
:103196002212957FEF64017065303B2CC23B900193
:1031A6009C04F0853E3FE53F75F010A424DAF974DF
:1031B6000F35F0FA7BFF129845AF3F128D1DE49054
:1031C6000190F090018F8032304133C24190019ED0
:1031D600E534F075F010A4241AF9741335F0FA7B6F
:1031E600FF12984590019EE0FF128B1A90019C7485
:1031F60002F0E4900190F090018F7405F022C23B3A
:10320600C24112957FEF64017069304A66120096DA
:10321600C239C24A90004EE0FFC39415505574D28D
:103226002FF582E43400F583E0FFA248E4336F70A3
:1032360042A248924990004EE0900191F090004FD2
:10324600E0900192F090004DE0900193F01271EB46
:10325600900193E0641F601B900191E0FF90019242
:10326600E0FD7C0012872EE4900190F090018F74AF
:1032760002F022C24A22E4900190F090018FF022DF
:103CFB00900190E070127BFF7A0F799412984590A7
:103D0B0001907401F0027ABB900190E06401706045
:103D1B00900000E060030241ED90008EE090000CFB
:103D2B00F09000B8E09001A3F090019CE0B4011278
:103D3B00AF3F129AC2E53F75F010A424DAF9740F65
:103D4B00802090019CE0640260030241ED90019E93
:103D5B00E0FF121E5890019EE075F010A4241AF992
:103D6B00741335F0FA7BFF12987A9001900241DDC3
:103D7B00900190E064026003023E0B129BEC205B0F
:103D8B00089000B8E07002800C9000B8E0600B90D7
:103D9B0001A3E07005127AC1805F305B329000B8EE
:103DAB00E09001A3F090019CE0B4010D303B0AE5DB
:103DBB003FB53E05C23B127ABB90019CE0B4020FAB
:103DCB0030410C90019EE0B53405C241127ABB1212
:103DDB00957FEF7003127AC19001E5E0B4010512F3
:103DEB007EF0803790008EE070030241ED90000C66
:103DFB00E060030241ED127EF09001907403F0221B
:103E0B00900190E0B40324205D189001C2E4F0A36C
:103E1B0074FFF09001BE7401F0D25D9001907404B8
:103E2B00F0227BFF7A0F797202987A900190E0640E
:103E3B0004702C127EFF127AC1E490019DF0900069
:103E4B005DE0600E90009FE0900009F09001900201
:103E5B0041359000A0E0900002F0120096801C907B
:103E6B000190E064056003023F8B900009E0701243
:103E7B001200969000A0E0900002F0900190740662
:103E8B00F02212957FEF64016003023F1712009638
:103E9B00303B39C23BE53F653E70030241ED90017B
:103EAB009C7401F0853E3FC239E53F75F010A424A8
:103EBB00DAF9740F35F0FA7BFF129845AF3F128D8C
:103ECB001DE4900190F090018F02413530413DC2CD
:103EDB004190019EE0653470030241ED90019EE537
:103EEB0034F075F010A4241AF9741335F0FA7BFF33
:103EFB0012984590019EE0FF128B1A90019C740260
:103F0B00F0E4900190F090018F024135C23BC24129
:103F1B0012957FEF64017065304A62120096C239C8
:103F2B00C24A90004EE0FFC39415505174D22FF546
:103F3B0082E43400F583E0FFA248E4336F703EA2C5
:103F4B0048924990004EE0900191F090004FE09024
:103F5B000192F090004DE0900193F01271EB900103
:103F6B0093E0641F6017900191E0FF900192E0FDD8
:103F7B007C0012872E90018F7402024025C24A22C8
:103F8B00900190E0640660030240A1900002E07093
:103F9B000F90008DE0900001F09001907407F022DB
:103FAB0012957FEF64017077303B35C23BE53F657F
:103FBB003E70030241ED90019C7401F0853E3FC2BF
:103FCB0039E53F75F010A424DAF9740F35F0FA7B5C
:103FDB00FF129845AF3F128D1D90018F7405803AEB
:103FEB0030413CC24190019EE0653470030241EDCB
:103FFB0090019EE534F075F010A4241AF974133572
:10400B00F0FA7BFF12984590019EE0FF128B1A90FD
:10401B00019C7402F090018F7405F0E402416BC2B5
:10402B003BC24112957FEF64017068304A65120004
:10403B0096C239C24A90004EE0FFC3941550547497
:10404B00D22FF582E43400F583E0FFA248E4336F0E
:10405B007041A248924990004EE0900191F090007F
:10406B004FE0900192F090004DE0900193F01271AF
:10407B00EB900193E0641F601A900191E0FF9001B7
:10408B0092E0FD7C0012872EE4900190F090018F5E
:10409B000241DDC24A22900190E0640760030241B5
:1040AB00E412957FEF6401600302413990008DE0CB
:1040BB00900001F0303B36C23BE53F653E7003029A
:1040CB0041ED90019C7401F0853E3FE53F75F0108A
:1040DB00A424DAF9740F35F0FA7BFF129845AF3F41
:1040EB00128D1DE4900190F090018F803D30413E88
:1040FB00C24190019EE0653470030241ED90019E38
:10410B00E534F075F010A4241AF9741335F0FA7B2A
:10411B00FF12984590019EE0FF128B1A90019C7440
:10412B0002F0E4900190F090018F7405F022C23BF5
:10413B00C241900001E0702D127AAF9000B4E060A4
:10414B0003127AD3127EFF900099E0FF789F7600DE
:10415B0008A6079001A27401F0C239E490018FF018
:10416B00900190F02212957FEF64017069304A66DE
:10417B00120096C239C24A90004EE0FFC39415500C
:10418B005574D22FF582E43400F583E0FFA248E4A6
:10419B00336F7042A248924990004EE0900191F02B
:1041AB0090004FE0900192F090004DE0900193F061
:1041BB001271EB900193E0641F601B900191E0FF83
:1041CB00900192E0FD7C0012872EE4900190F0901C
:1041DB00018F7402F022C24A22E4900190F0900108
:0341EB008FF02230
:104EA100900190E070469001E3E0900052F0900193
:104EB100E4E0900053F07BFF7A0F79A5129845E466
:104EC1009001E2F0900052E0FF900053E0FD7C0081
:104ED10012872E900052E024D2F582E43400F5834B
:104EE100E024FF92499001907401F022900190E03A
:104EF1006401704B900000E06003025293A249925A
:104F01004D9001E3E090015BF09001E4E090015CE1
:104F1100F090005BE090015DF012692490015EEF7A
:104F2100F0128693D23F12728D900082E09001A41C
:104F3100F090008EE090000CF0900190025283906E
:104F41000190E064026003025041129BEC305B105F
:104F5100304A0D900082E09001A4F0C24A127ABB5F
:104F610012957FEF7003127AC19001E5E0B4010C54
:104F7100E4F0127EF09001907404F0229001A4E01C
:104F81007008900082E06002800C90008EE060105A
:104F910090000CE0700A127EF09001907403F022F0
:104FA100787BE660030252933057030252939001DB
:104FB10097E07032A249924D9001E3E090015BF0DD
:104FC1009001E4E090015CF090005BE090015DF005
:104FD10012692490015EEFF0128693D23F12728D16
:104FE1009001970252831283AEEF6401704F9001DA
:104FF10058E0FF2442F582E43401F583E090015B3F
:10500100F0742D2FF582E43401F583E090015CF01A
:10501100900158E090015DF012640490015EEFF0A0
:1050210090015BE024D2F582E43400F583E024FFB3
:10503100924D128693D23F12728D0250EE0250EEC3
:10504100900190E0B40323205D179001C2E4F0A326
:1050510074FFF09001BE7401F0D25D900190740470
:10506100F07BFF7A0F797202987A900190E06404E4
:105071007049127EFF127AC1787BE6600302529377
:10508100305703025293A249924D900191E0900151
:105091005BF0900192E090015CF090015D741FF073
:1050A100129B7090015EEFF012869390019774034A
:1050B100F012728D9001907405F022900190E0FF42
:1050C10064057030787BE660030252933057030227
:1050D1005293900197E0700F90008DE0900001F0E5
:1050E1009001907406F022787B7628D25790019730
:1050F100E014F022EF6406600302528A900001E09E
:10510100702A127AAF9000B4E06003127AD3127E53
:10511100FF900099E0FF789F760008A6079001A212
:105121007401F0C239E490018FF0806912957FEF2C
:1051310064017066303B2DC23B90019C04F0853EBA
:105141003FC239E53F75F010A424DAF9740F35F048
:10515100FA7BFF129845AF3F128D1D90018F7405A8
:10516100F0E48031304133C24190019EE534F07565
:10517100F010A4241AF9741335F0FA7BFF12984544
:1051810090019EE0FF128B1A90019C7402F0900135
:105191008F7405F0E4900190F022C23BC241129558
:1051A1007FEF6401600302528790008DE09000015F
:1051B100F0204A03025287120096C239C24A900176
:1051C10091E0FF90004EE0FEB5071290004FE0FF26
:1051D100900192E0B50706E4900195F022EEC394A8
:1051E10015400302528790004EE0FF24D2F582E47D
:1051F1003400F583E0FEA248E4336E600302528777
:10520100900195E0FE701BA2489249900194EFF045
:1052110090004FE0900195F090004DE0900196F0E4
:10522100806490004EE0FF6E705CA248924990014C
:1052310091EFF090004FE0900192F090004DE090DE
:105241000193F01271EB900193E0641F60389001BB
:1052510091E0FFC39415502E74D22FF582E43400EF
:10526100F583E0FFA249E433B5071B900191E0FF0C
:10527100900192E0FD7C0012872EE4900190F09065
:10528100018F7402F022C24A22E4900190F0900151
:035291008FF02279
:1037EE00900190E0706390005BE0900052F09000CA
:1037FE005374FEF09001E2E0B4011D9001E4E0F597
:10380E003F7BFF7A0F79B61298459001E4E0FF12E4
:10381E008D1D90019C7401F09001E2E0B4021F90A6
:10382E0001E4E090019EF07BFF7A0F79C912984572
:10383E009001E4E0FF128B1A90019C7402F0E49068
:10384E0001E2F090019004F022900190E06401708A
:10385E0058900000E06003023CFA90008EE0900069
:10386E000CF090019CE0B40112AF3F129AC2E53FFA
:10387E0075F010A424DAF9740F802090019CE06496
:10388E00026003023CFA90019EE0FF121E58900166
:10389E009EE075F010A4241AF9741335F0FA7BFF2C
:1038AE0012987A900190023CEA900190E0640270C6
:1038BE0061129BEC305B2A90019CE0B4010D303B11
:1038CE000AE53FB53E05C23B127ABB90019CE0B4BF
:1038DE00020F30410C90019EE0B53405C241127AC0
:1038EE00BB12957FEF7003127AC19001E5E0B4012F
:1038FE0005127EF0803790008EE07003023CFA9045
:10390E00000CE06003023CFA127EF090019074030A
:10391E00F022900190E0B40324205D189001C2E4DF
:10392E00F0A374FFF09001BE7401F0D25D9001908F
:10393E007404F0227BFF7A0F797202987A900190CC
:10394E00E064047027127EFF127AC190005DE06081
:10395E000E90009FE0900009F0900190023C75904F
:10396E0000A0E0900002F0120096801C900190E002
:10397E0064056003023A9B900009E07012120096F3
:10398E009000A0E0900002F09001907406F02212D8
:10399E00957FEF64016003023A27120096303B399F
:1039AE00C23BE53F653E7003023CFA90019C7401F8
:1039BE00F0853E3FC239E53F75F010A424DAF97464
:1039CE000F35F0FA7BFF129845AF3F128D1DE49034
:1039DE000190F090018F023C7530413DC241900143
:1039EE009EE065347003023CFA90019EE534F0755A
:1039FE00F010A4241AF9741335F0FA7BFF129845CF
:103A0E0090019EE0FF128B1A90019C7402F0E490DC
:103A1E000190F090018F023C75C23BC24112957F1E
:103A2E00EF64017065304A62120096C239C24A9044
:103A3E00004EE0FFC39415505174D22FF582E4343A
:103A4E0000F583E0FFA248E4336F703EA24892492E
:103A5E0090004EE0900191F090004FE0900192F0B6
:103A6E0090004DE0900193F01271EB900193E064A1
:103A7E001F6017900191E0FF900192E0FD7C001213
:103A8E00872E90018F7402023B35C24A229001901C
:103A9E00E064066003023BB1900002E0700F9000FC
:103AAE008DE0900001F09001907407F02212957F46
:103ABE00EF64017077303B35C23BE53F653E7003E6
:103ACE00023CFA90019C7401F0853E3FC239E53FFD
:103ADE0075F010A424DAF9740F35F0FA7BFF129802
:103AEE0045AF3F128D1D90018F7405803A30413CD9
:103AFE00C24190019EE065347003023CFA90019E33
:103B0E00E534F075F010A4241AF9741335F0FA7B2D
:103B1E00FF12984590019EE0FF128B1A90019C7443
:103B2E0002F090018F7405F0E4023BE7C23BC24104
:103B3E0012957FEF64017068304A65120096C239A3
:103B4E00C24A90004EE0FFC39415505474D22FF524
:103B5E0082E43400F583E0FFA248E4336F7041A2A3
:103B6E0048924990004EE0900191F090004FE09005
:103B7E000192F090004DE0900193F01271EB9001E4
:103B8E0093E0641F601A900191E0FF900192E0FDB6
:103B9E007C0012872EE4900190F090018F023CEA97
:103BAE00C24A22900190E064076003023CF190004B
:103BBE0001E0702A127AAF9000B4E06003127AD35B
:103BCE00900099E0FF789F760008A6079001A274F6
:103BDE0001F0C239E490018FF0900190F02212951D
:103BEE007FEF64016003023C7990008DE09000014C
:103BFE00F0303B36C23BE53F653E7003023CFA9027
:103C0E00019C7401F0853E3FE53F75F010A424DA67
:103C1E00F9740F35F0FA7BFF129845AF3F128D1DE8
:103C2E00E4900190F090018F803D30413EC2419072
:103C3E00019EE065347003023CFA90019EE534F07B
:103C4E0075F010A4241AF9741335F0FA7BFF12984C
:103C5E004590019EE0FF128B1A90019C7402F0E4D5
:103C6E00900190F090018F7405F022C23BC2411278
:103C7E00957FEF64017069304A66120096C239C2B0
:103C8E004A90004EE0FFC39415505574D22FF58222
:103C9E00E43400F583E0FFA248E4336F7042A2489B
:103CAE00924990004EE0900191F090004FE090010B
:103CBE0092F090004DE0900193F01271EB90019311
:103CCE00E0641F601B900191E0FF900192E0FD7C8B
:103CDE000012872EE4900190F090018F7402F02272
:0D3CEE00C24A22E4900190F090018FF02274
:1000A600202020202020202020202020202020204A
:1000B6005245504541544552204E554D42455220D9
:1000C6002020202020202020203120746F20323054
:1000D600202053495445204E554D4245522020205C
:1000E6002020202020202020203120746F20393924
:1000F6008202001101021501148202011103041586
:1001060001632020202020202020202020202020C5
:1001160020202020202020202020202020202020D9
:10012600202020434F5552544553592042454550AF
:100136002020204354435353204F4E2048414E47DE
:10014600202020205553455220454E41424C452003
:10015600202020205245534552564520544F4E45A7
:10016600202020204E4554574F524B204D4F44459A
:100176002020204E4554574F524B204E554D424558
:100186005220202020202020202020202020202037
:100196002020202020202020202020202020202059
:1001A6002020202020202020202020202020202049
:1001B6002020202020202020202020202020202039
:1001C6002020202020202020202020202020313DFB
:1001D600454E2020202020202020202020204D4F6A
:1001E6004445202020202020202020202020544F5D
:1001F6004E4564010011020C150001640200110352
:100206000C15000164040011040C150001640800BB
:1002160011050C15000164100011060D150002C829
:10022600030111070A190101202020202020202087
:1002360020202020202020202020202020202020B8
:10024600202020202020202020434F555254455363
:100256005920424545502020204354435353204FB4
:100266004E2048414E4720202020555345522045D8
:100276004E41424C4520202020205245534552569F
:100286004520544F4E45202020204E4554574F526E
:100296004B204D4F44452020204E4554574F524B3E
:1002A600204E554D4245522020202020202020203F
:1002B6002020202020202020202020202020202038
:1002C6002020202020202020202020202020202028
:1002D6002020202020202020202020202020202018
:1002E6002020202020202020202020202020202008
:1002F60020202020313D454E202020202020202077
:10030600202020204D4F4445202020202020202042
:1003160020202020544F4E4564010011020C150088
:100326000164020011030C15000164040011040CA1
:1003360015000164080011050C1500016410001178
:10034600060D150001C8030111070A190101202035
:100356002020202020202020202020202020202097
:100366002020202020202020202020202020204364
:100376004F55525445535920424545502020202080
:100386005553455220454E41424C4520202020439E
:10039600524F535320544F4E45204D4F4445204312
:1003A600544353532F4443532043524F5353202017
:1003B6004E4554574F524B204D4F44452020204E1A
:1003C6004554574F524B204E554D42455220202002
:1003D6002020202020202020202020202020202017
:1003E60020202020202020202020313D454E202086
:1003F600202020202020202020204D4F4445202052
:1004060020202020202020202020544F4E45202030
:1004160020202020202020202020202020206401B1
:1004260000110209150001640200110309150001FB
:1004360064040011060A150001C8030111070C190E
:1004460001012020202020202020202020202020E4
:100456002020202020202020202020202020202096
:10046600202001010101010101010100000000003D
:100476000000000000000000000000000000000076
:100486000000000000000000000000000000000066
:100496000000000000000000000000000000000056
:1004A6000000000000000000000000000000000046
:1004B60000000000000000000000000020202020B6
:1004C6002020202020202020202020202020202026
:1004D6002020202020202020202020200101010192
:1004E6000101010101000000000000000000000001
:1004F60000000000000000000000000000000000F6
:1005060000000000000000000000000000000000E5
:1005160000000000000000000000000000000000D5
:1005260000000000000000000000000000000000C5
:100536000000000000002020202020202020202075
:1005460020202020202020202020202020202020A5
:1005560020202020202001010101010101010120AC
:100566002020202020202020202020202020202085
:100576002020202020202020202020202020202075
:1005860054454C434F2050524F4752414D20202056
:10059600524144494F2050524F4752414D2020204E
:1005A60050484F4E452050524F4752414D20202033
:1005B600434F4D50552050524F4752414D20202019
:1005C6002041434345535320434F44452020204474
:1005D600544D462054454C434F204C4556454C44BB
:1005E600544D4620524144494F204C4556454C42B5
:1005F60045455020524144494F204C4556454C42B2
:100606004545502054454C434F204C4556454C4398
:1006160057494420524144494F204C4556454C5673
:100626004F49434520524144494F204C45564C566C
:100636004F4943452054454C434F204C45564C505A
:1006460041474520524144494F204C4556454C436D
:100656005443535320524144494F204C45564C4431
:10066600435320524144494F204C4556454C204C5B
:10067600545220524144494F204C4556454C205235
:10068600505420524144494F204C4556454C205425
:10069600454C434F20524144494F204C45564C52FD
:1006A6004144494F2054454C434F204C45564C52EB
:1006B6004144494F204C494D4954204C45564C2005
:1006C600434F53204F5220535155454C4348202009
:1006D60020434F5320504F4C4152495459202043F8
:1006E6004F53205452494747455220564F4C544386
:1006F6004F5320414351554953542054494D454386
:100706004F532052454C454153452054494D4520B1
:1007160053454E534520504F4C415249545920534E
:10072600454E205452494747455220564F4C545344
:10073600454E20414351554953542054494D455344
:10074600454E2052454C454153452054494D452080
:100756004C545220484F4C442044454C415920505B
:100766005454205455524E4F46462054494D4552F6
:10077600455045415445522054494D454F55542006
:1007860020414E54492D4B45524348554E4B20204F
:1007960020535155454C4348205441494C20202074
:1007A60043544353532F44435320484F4C44204310
:1007B600524F535320425553592044454C415943B7
:1007C600524F5353204255535920484F4C442020F2
:1007D600204C54522053594E432042495420202045
:1007E600414456414E43454420204C4F434B202024
:1007F60020202020202020202020202020202020F3
:1008060020202020202020202020202020202020E2
:1008160020202020202020202020202020202020D2
:1008260020202020202020202020202020202020C2
:100836002020202020202020202020313D454E2031
:1008460020202020202020202020524154494F20C3
:1008560020202020202020202020303D434F5320E0
:1008660020202020202020202020313D504F5320C2
:10087600202020202020202020202031204D532001
:10088600202020202020202020203130204D5320E1
:10089600202020202020202020313030204D5320C1
:1008A60020202020202020202020202053454320C7
:1008B600202020202020202020313D534B4950204D
:1008C6002020202020202020202020202020202022
:1008D6002020202020202020202020202020202012
:1008E6005052494F52495459204C4556454C2020A8
:1008F6004C545220454E434F444520504F4C2020E7
:100906004C5452204445434F444520504F4C2020E0
:10091600205445535420494420434F444520204900
:10092600444C45204D45535341474520544D522094
:100936002020204152454120424954202020202099
:100946004D4153544552204F5220534C4156452059
:1009560044435320454E434F444520504F4C20209E
:10096600444353204445434F444520504F4C202098
:10097600434F5552544553592044454C4159202024
:10098600202048414E472054494D452020202043F1
:100996004152524945522044524F5020444C59200E
:1009A600204143434553532044454C41592020534D
:1009B600544154494F4E204944204D4F4445202030
:1009C600564F494345204F52204357494420202043
:1009D60020494420494E54455256414C202020205F
:1009E6002020435749442053504545442020202089
:1009F60043574944204652455155454E43592020B8
:100A06002043574944204D45535341474520202014
:100A16005455524E5F4F4E2044454C41592020209C
:100A26005455524E5F4F46462044454C415920206E
:100A360042454550204652455155454E4359205250
:100A4600455045415445522044495341424C452066
:100A56004155582052454C4159204D4F4445202080
:100A660043524F53532042555359204D4F4445202E
:100A76005245504541544552204741494E20202079
:100A86002054454C434F204741494E202020204EBC
:100A96004554574F524B2048414E4754494D4520E7
:100AA6002020202020202020204C4556454C202068
:100AB600202020202020202020303D4E4F524D2047
:100AC6002020202020202020202020434F44452085
:100AD6002020202020202020202020415245412077
:100AE60020202020202020303D4D415354455220C7
:100AF600202020202020202020202031204D53207F
:100B0600202020202020202020203130204D53205E
:100B1600202020202020202020313030204D53203E
:100B26002020202020202020203130205345432023
:100B36002020202020202020202031204D494E201A
:100B460020202020202020202020204D4F444520FA
:100B56002020202020202020303D564F494345208C
:100B660020202020202020202020204652455120D1
:100B76002020202020202020202020313D454E20EE
:100B860020414C41524D20434F554E5420202020A9
:100B9600524553544F524520434F554E5420202022
:100BA6002020494E54455256414C202020202020DA
:100BB6004E4554574F524B20434F44452020204921
:100BC6004E544552434F4E4E454354204D4F444E8E
:100BD6004554574F524B20494E414354495645823E
:100BE600010011022D15000182010111032D1500CE
:100BF6000182010211042D15000182010311052D48
:100C060015000178060411060119010182030A1173
:100C1600072E1500FF82030B11082E1500FF820315
:100C26000C11092E1500FF82030D110A2E1500FF67
:100C360082030E110B2E1500FF82030F110C2E15C9
:100C460000FF820310110D2E1500FF820311110EF5
:100C56002E1500FF820312110F2E1500FF820313BB
:100C660011102E1500FF82031411112E1500FF829C
:100C7600031511122E1500FF82031611132E1500EF
:100C8600FF82031711142E1500FF82031811152E6B
:100C96001500FF82011911162F15000182011A1184
:100CA600173015000182031B11182E1500FF820252
:100CB6001C11193115006382021D111A32150063C9
:100CC60082011E111B3015000182031F111C2E15F7
:100CD60000FF820220111D31150063820221111EC0
:100CE60032150063820222111F3315026382032329
:100CF6001120321501FF8203241121341502FF82CF
:100D060002251122331500638202261123321500B3
:100D160063820227112433150363820228112532C8
:100D26001500638203291126331500FA82012A1160
:100D3600273515000182012B11385415010982014E
:100D46002C11395515000182012D113A5515000156
:100D560082032E113B561501FA82032F113C5C15B6
:100D660000FF820130113D57150001820131113E0D
:100D760058150001820132113F55160001820133D8
:100D860011405515000182023411415A1500638243
:100D9600023511425B15006382023611435A150073
:100DA6006382023711445A15006382013811455E89
:100DB60015000182013911465F15000182023A11C0
:100DC600475D15006382023B114859150463820290
:100DD6003C114960150114BE0A3D114A5611000026
:100DE600820247114B5A150063820248114D601565
:100DF6000114820149114E5E15000282014A114F0B
:100E06006115000182014B11505E15000482014CF0
:100E160011515415010982014D11525415010982CF
:100E2600024E11533415006382014F116201150001
:100E36000982015011630115000982025111645D96
:100E4600150163C803521165011501018201541190
:100E5600665E1500028203551167341500FF010115
:100E66000200000200000200000000000001010173
:100E76003132333435361432320532FFFFFF191959
:100E8600196464C8FF000180000A0180000A1E1A66
:100E9600B400001E1E1E0001000002010001000039
:100EA6000A1E630A000100050520202020202020BC
:100EB6002020200A050000000101140000010000A6
:020EC60000002A
:109845008B738A7489757F01127ED6E49000E7F0E8
:109855009000E7E0FFC39410501AAB73AA74A97582
:109865008F82758300128606FF127EA79000E7E0BF
:0598750004F080DC227C
:106C4B008B738A7489759001F9E0B41100400302CB
:106C5B006DC8906C64F8282873026C97026C9F02C5
:106C6B006CAF026CC2026CD5026CE8026CFB026D5D
:106C7B000E026D21026D34026D46026D58026D6A73
:106C8B00026D7C026D8E026DA0026DB27F01127ED1
:106C9B00D6026DC2AB73AA74A9751285EDFF127E75
:106CAB00A7026DC2AB73AA74A97590000112860678
:106CBB00FF127EA7026DC2AB73AA74A97590000276
:106CCB00128606FF127EA7026DC2AB73AA74A9755A
:106CDB00900003128606FF127EA7026DC2AB73AA49
:106CEB0074A975900004128606FF127EA7026DC26E
:106CFB00AB73AA74A975900005128606FF127EA7C6
:106D0B00026DC2AB73AA74A975900006128606FFBA
:106D1B00127EA7026DC2AB73AA74A97590000712FD
:106D2B008606FF127EA7026DC2AB73AA74A975907B
:106D3B000008128606FF127EA7807CAB73AA74A98B
:106D4B0075900009128606FF127EA7806AAB73AAA4
:106D5B0074A97590000A128606FF127EA78058ABA5
:106D6B0073AA74A97590000B128606FF127EA7807A
:106D7B0046AB73AA74A97590000C128606FF127E9F
:106D8B00A78034AB73AA74A97590000D128606FF09
:106D9B00127EA78022AB73AA74A97590000E12867F
:106DAB0006FF127EA78010AB73AA74A97590000F13
:0E6DBB00128606FF127EA79001F9E004F02276
:10987A008B738A7489757F11127ED6E49000E7F0A3
:10988A009000E7E0FFC39410501AAB73AA74A9754D
:10989A008F82758300128606FF127EA79000E7E08A
:0598AA0004F080DC2247
:104A9000E49001A8F0A3F09001AAF09000EBF0A33D
:104AA000F09000ECE02400F582E43404F583E4F0B7
:104AB0009000ECE004F070069000EBE004F0900051
:104AC000EBE07004A3E0648070D7E49000E7F0901E
:104AD00000E7E0FFC394024003024B61EF900E64D5
:104AE00093FF9001AAE0FE04F074002EF582E434F6
:104AF00004F583EFF09001AAE06480705B9001A858
:104B0000E0FEA3E07807C333CE33CED8F9FF7C04B0
:104B10007D0012752EE49000EBF0A3F09000ECE025
:104B20002400F582E43404F583E4F09000ECE00422
:104B3000F070069000EBE004F09000EBE07004A34E
:104B4000E0648070D7E49001AAF09001A9E004F03D
:104B500070069001A8E004F09000E7E004F0024A3B
:104B6000CFE49000EAF0E49000E8F0A3F0E49000D5
:104B7000E7F09000E7E0FFC394034003024C04EF2A
:104B8000900E6693FF9001AAE0FE04F074002EF5EB
:104B900082E43404F583EFF09001AAE06480705B56
:104BA0009001A8E0FEA3E07807C333CE33CED8F956
:104BB000FF7C047D0012752EE49000EBF0A3F090D2
:104BC00000ECE02400F582E43404F583E4F0900086
:104BD000ECE004F070069000EBE004F09000EBE0F5
:104BE0007004A3E0648070D7E49001AAF09001A95A
:104BF000E004F070069001A8E004F09000E7E00403
:104C0000F0024B729000E9E004F070069000E8E0DA
:104C100004F0C39000E9E094339000E8E094005081
:104C200003024B6D9000EAE004F0E0C394145003DB
:104C3000024B66E49000EAF0E49000E8F0A3F0E4B0
:104C40009000E7F09000E7E0FFC394034003024CBC
:104C5000D6EF900E6993FF9001AAE0FE04F0740075
:104C60002EF582E43404F583EFF09001AAE064802D
:104C7000705B9001A8E0FEA3E07807C333CE33CE8B
:104C8000D8F9FF7C047D0012752EE49000EBF0A3B0
:104C9000F09000ECE02400F582E43404F583E4F0C5
:104CA0009000ECE004F070069000EBE004F090005F
:104CB000EBE07004A3E0648070D7E49001AAF09068
:104CC00001A9E004F070069001A8E004F09000E76C
:104CD000E004F0024C449000E9E004F0700690001B
:104CE000E8E004F0C39000E9E094709000E8E094FC
:104CF000005003024C3F9000EAE004F0E0C394143B
:104D00005003024C38E49000E8F0A3F0E49000E790
:104D1000F09000E7E0FFC394034003024DA3EF903F
:104D20000E6C93FF9001AAE0FE04F074002EF58251
:104D3000E43404F583EFF09001AAE06480705B90A6
:104D400001A8E0FEA3E07807C333CE33CED8F9FF45
:104D50007C047D0012752EE49000EBF0A3F090002F
:104D6000ECE02400F582E43404F583E4F09000ECF8
:104D7000E004F070069000EBE004F09000EBE070CF
:104D800004A3E0648070D7E49001AAF09001A9E048
:104D900004F070069001A8E004F09000E7E004F051
:104DA000024D119000E9E004F070069000E8E00484
:104DB000F0C39000E9E094889000E8E09413500379
:104DC000024D0C8000E49000E8F0A3F0E49000E7CE
:104DD000F09000E7E0FFC394564003024E63EF906B
:104DE0000E7293FF9001AAE0FE04F074002EF5828B
:104DF000E43404F583EFF09001AAE06480705B90E6
:104E000001A8E0FEA3E07807C333CE33CED8F9FF84
:104E10007C047D0012752EE49000EBF0A3F090006E
:104E2000ECE02400F582E43404F583E4F09000EC37
:104E3000E004F070069000EBE004F09000EBE0700E
:104E400004A3E0648070D7E49001AAF09001A9E087
:104E500004F070069001A8E004F09000E7E004F090
:104E6000024DD19000E9E004F070069000E8E00403
:104E7000F0C39000E9E094149000E8E0940050033F
:104E8000024DCC9001A8E0FEA3E07807C333CE33F7
:104E9000CED8F9FF7C047D0012752E127EF0027EC2
:014EA000FF12
:109BA900E4900059F0A3F0FFFE1274D790005BEF28
:029BB900F02298
:1088590075530175540075556AE49001F6F0A3F05B
:108869009001F6E0FAA3E0FBC39456EA9400504065
:1088790090005BE075F056A42478FFE5F03460CFF2
:108889002BCF3AFE900059F0A3EFF01274D7AB53F7
:108899000555E555AA547002055414F9EF128633AB
:1088A9009001F7E004F070B89001F6E004F080B0B0
:1088B90090009BE07004D2588002C258900097E063
:1088C90024FF924F900096E024FF924490009DE08F
:1088D90024FF924E90009CE024FF924590007CE09A
:0288E900F52D6B
:0188EB00226A
:1090E4007553017554007555BFE49001F6F0A3F073
:1090F4009001F6E0FEA3E0FFC39414EE9400503B0D
:109104007C007D56128645EF24F9FFEE3460FE9014
:109114000059F0A3EFF01274D7AB530555E555AAE7
:10912400547002055414F9EF1286339001F7E004E9
:0B913400F070BD9001F6E004F080B583
:01913F00220D
:109140007553017554007555D3E49001F6F0A3F002
:109150009001F6E0FEA3E0FFC39414EE9400503BB0
:109160007C007D56128645EF24FEFFEE3460FE90B3
:109170000059F0A3EFF01274D7AB530555E555AA8B
:10918000547002055414F9EF1286339001F7E0048D
:0B919000F070BD9001F6E004F080B527
:01919B0022B1
:108D1D008F73E49000E7F09000E7E0FBC3940350FD
:108D2D003E90005BE075F099A42469FDE5F034FFF9
:108D3D00FCE57375F003A42DFFE5F03CFEEB7C0024
:108D4D002FFFEC3EFE1274D79000E7E02461F58210
:108D5D00E43400F583EFF09000E7E004F080B89084
:108D6D000061E0FE540190005CF0EE540290005D55
:108D7D00F0900061E0540490005EF0EE5408900015
:0D8D8D005FF0900061E05410900060F02253
:108B1A008F73E49000E7F09000E7E0FBC394035002
:108B2A004490005BE0FF7E007C017D50128645EF99
:108B3A0024A6FDEE340AFCE57375F003A42DFFE5C7
:108B4A00F03CFEEB7C002FFFEC3EFE1274D7900047
:108B5A00E7E02461F582E43400F583EFF09000E762
:108B6A00E004F080B2900061E0FE540190005CF0F5
:108B7A00EE540290005DF0900061E0540490005EB3
:108B8A00F0EE540890005FF0900061E054109000FD
:038B9A0060F02266
:06872E008F738C748D7541
:10873400E49001F6F0A3F0E57524FFFFE57434FF3F
:10874400FE7C007D03128645AA06AB07AE73E57373
:1087540025E0CE75F0EEA4FFE5F02EFEEF2448FFF1
:10876400EE3423CF2BCF3AFE9001F7E02FFF900198
:10877400F6E03EFE1274D79001F7E02461F582E43E
:108784003400F583EFF09001F7E004F070069001F7
:10879400F6E004F0C39001F7E094039001F6E0944E
:1087A400004094900061E0FE5401900067F0EE54A4
:0F87B40002900068F0900061E05404900069F0BA
:0187C3002293
:109A83002020202020534C415645202020202020F8
:109A930020202020204D41535445522020202020B7
:0E9BFC00127E04127EF0127EFF7F01027ED6E2
:1098AF009000037414F0127EF0900003E070FA90B1
:1098BF00009BE07BFF60067A9A798380047A9A791D
:1098CF009312987A9000037414F0127EF0900003B4
:0498DF00E070FA2219
:10784A00C0D0C0E0C0F0C000A88475840FE55854C9
:10785A0007B4000D85E8F0A2F09220A2F1922180EF
:10786A0076B4010D85E8F0A2F09222A2F19223806B
:10787A0066B4020D85E8F0A2F09224A2F192258066
:10788A0056B4030D85E8F0A2F09226A2F192278061
:10789A0046B4040D85E8F0A2F09218A2F19219807C
:1078AA0036B4050D85E8F0A2F0921AA2F1921B8077
:1078BA0026B4060D85E8F0A2F0921CA2F1921D8072
:1078CA001685E8F0A2F0921EA2F1921F7558FF8564
:1078DA00231E85241FD260055875590A8884D00052
:1078EA00D0F0D0E0D0D032205F0122D2B7E55A548E
:1078FA0007B4000AA22F92F7A22E92F6805EB40174
:10790A000AA22D92F7A22C92F68051B4020AA22B57
:10791A0092F7A22A92F68044B4030AA22992F7A205
:10792A002892F68037B4040AA23792F7A23692F662
:10793A00802AB4050AA23592F7A23492F6801DB4C1
:10794A00060AA23392F7A23292F68010B40721A255
:10795A003192F7A23092F6C25F755AFF055A7584C2
:10796A000F85E8E0A2F692E6A2F792E7F5E8C2B739
:01797A0022EA
:109084009001D2E0FFEF12866D90B20090B601908D
:10909400BA0290BE0390C20490C60590CA0690CE50
:1090A4000790D20890D60990DA0A000090DE128E5A
:1090B40082221287C4221292A022128D9A22128135
:1090C4000D2212853D22127F0E2212967C221293CB
:1090D4004722125E9722126070229001D2E4F0229D
:108E82003061669001D3E4F0C261E55612866D8EC0
:108E9200B0478EB7488EBE498EC54A8ECC4B8ED314
:108EA2004C8EDA4D8EE14E8EE54F00008EEB900136
:108EB200D27401F0229001D27402F0229001D27495
:108EC20003F0229001D27404F0229001D27405F0D2
:108ED200229001D27406F0229001D27407F022127D
:0A8EE2009B45229001D27408F02293
:1087C4009001D3E0FFEF70189001DA7401F090018A
:1087D400DB7401F09001D27409F09001D3E4F0222B
:1087E4009001D3E0FFEFB401189001DA7401F09026
:1087F40001DB7402F09001D2740AF09001D3E4F02A
:10880400229001D3E0FFEF640270499001D8E4F0B4
:10881400A3E4F09001D8E475F001128657AFF0FE9E
:10882400EF4E60269001D4E475F001128657AFF044
:10883400FE9001D8E0FCA3E0FD74002DF5827408DD
:108844003CF583E0FD12749680C97F011200869086
:0588540001D2E4F02256
:1092A0009001D3E0FFEF70189001DA7402F09001A2
:1092B000DB7401F09001D27409F09001D3E4F02244
:1092C0009001D3E0FFEFB401189001DA7402F0903E
:1092D00001DB7402F09001D2740AF09001D3E4F043
:1092E000229001D3E0FFEFB4020A7F0112008690C2
:0592F00001D2E4F022B0
:108D9A009001D3E0FFEF70189001DA7403F09001AC
:108DAA00DB7401F09001D27409F09001D3E4F0224F
:108DBA009001D3E0FFEFB401189001DA7403F09048
:108DCA0001DB7402F09001D27409F09001D3E4F04F
:108DDA00229001D3E0FFEFB4021C205F2F9001D450
:108DEA00E0FEA3E0FF9001C2EEF0A3EFF0D25F90A5
:108DFA0001D3E004F0229001D3E0FFEFB4030D2089
:0D8E0A005F0A7F011200869001D2E4F02281
:10810D009001D3E0FFEF70189001DA7404F0900144
:10811D00DB7401F09001D27409F09001D3E4F022E8
:10812D009001D3E0FFEF640170749001D6E0FEA3DF
:10813D00E0FF9001D8EEF0A3EFF09001E0E4F0A3A2
:10814D00E4F09001D8E4F0A3E4F09001D8E475F0E8
:10815D0001128657AFF0FEEF4E602B9001D4E475FF
:10816D00F001128657AFF0FE1274D79001E0E4755E
:10817D00F001128657ADF0FC74002DF58274083CA9
:10818D00F583EFF080C4900800E0FF1200869001A7
:10819D00E0E4F0A37401F09001D3E004F02290012B
:1081AD00D3E0FFEF6402703F30624D9001E0E47563
:1081BD00F001128657AFF0FE74002FF58274083E61
:1081CD00F583E0FF1200869001D6E0FEA3E0FF905C
:1081DD0001E0E0FCA3E0FDC3ED9FEC9E50022222E6
:1081ED009001D3E004F0229001D3E0FFEFB4030837
:0981FD003062059001D2E4F02289
:10853D009001D3E0FFEF70189001DA7405F090010F
:10854D00DB7401F09001D27409F09001D3E4F022B4
:10855D009001D3E0FFEFB4012C9001D6E0FEA3E033
:10856D00FF128C9E900800E0FF1200869001D674D9
:10857D0004F0A3E4F09001E0E4F0A37401F09001A5
:10858D00D3E004F0229001D3E0FFEF6402703F309E
:10859D00624D9001E0E475F001128657AFF0FE7464
:1085AD00002FF58274083EF583E0FF1200869001DE
:1085BD00D6E0FEA3E0FF9001E0E0FCA3E0FDC3EDFB
:1085CD009FEC9E500222229001D3E004F0229001F4
:1085DD00D3E0FFEFB403083062059001D2E4F0223E
:107F0E009001D3E0FFEF70189001DA7406F0900143
:107F1E00DB7401F09001D27409F09001D3E4F022E9
:107F2E009001D3E0FFEFB401289001C27430F0A3AA
:107F3E00E4F09001D4E0FEA3E0FF9001C4EEF0A3C4
:107F4E00EFF09001BE7402F0D25F9001D3E004F026
:107F5E00229001D3E0FFEFB4020D305F0302800FD9
:107F6E009001D3E004F0229001D3E0FFEFB4030DB3
:107F7E00205E0302800F9001D3E004F0229001D323
:107F8E00E0FFEFB40421900800E0FF12008690019C
:107F9E00D67404F0A3E4F09001E0E4F0A37401F0D1
:107FAE009001D3E004F0229001D3E0FFEF6405705E
:107FBE003F30624D9001E0E475F001128657AFF04C
:107FCE00FE74002FF58274083EF583E0FF120086E2
:107FDE009001D6E0FEA3E0FF9001E0E0FCA3E0FDFF
:107FEE00C3ED9FEC9E500222229001D3E004F022BA
:107FFE009001D3E0FFEFB406083062059001D2E4A1
:02800E00F0225E
:10967C009001D3E0FFEF7011C2619001D47402F03D
:10968C00A3E4F09001D3E004F09001D3E0FFEFB439
:10969C00011A205D179001D4E0FEA3E0FF9001C2F7
:0D96AC00EEF0A3EFF0D25D9001D2E4F022C9
:109347009001D3E0FFEF7024306144C2619001D4F3
:109357007401F0A3E4F0AF567E009001D5E02FF042
:109367009001D4E03EF09001D3E004F09001D3E007
:10937700FFEFB4011A205D179001D4E0FEA3E0FFD0
:109387009001C2EEF0A3EFF0D25D9001D2E4F0229B
:105E970020610302606FC2619001D3E0FFEF7016CB
:105EA700AF56128A0D7E009001D4EEF0A3EFF0906A
:105EB70001D3E004F0229001D3E0FFEFB401389062
:105EC70001D4E0FEA3E0FFEFC4F8540FC868FFEE6B
:105ED700C454F048FE9001D4EEF0A3EFF0AF561291
:105EE7008A0D7E009001D5E02FF09001D4E03EF0BE
:105EF7009001D3E004F0229001D3E0FFEFB4023821
:105F07009001D4E0FEA3E0FFEFC4F8540FC868FF88
:105F1700EEC454F048FE9001D4EEF0A3EFF0AF5674
:105F2700128A0D7E009001D5E02FF09001D4E03E5B
:105F3700F09001D3E004F0229001D3E0FFEFB40327
:105F4700389001D4E0FEA3E0FFEFC4F8540FC8680F
:105F5700FFEEC454F048FE9001D4EEF0A3EFF0AF8B
:105F670056128A0D7E009001D5E02FF09001D4E003
:105F77003EF09001D3E004F0229001D3E0FFEFB4AC
:105F87000416AF56128A0D7E009001D6EEF0A3EFED
:105F9700F09001D3E004F0229001D3E0FFEFB405C5
:105FA700389001D6E0FEA3E0FFEFC4F8540FC868AD
:105FB700FFEEC454F048FE9001D6EEF0A3EFF0AF29
:105FC70056128A0D7E009001D7E02FF09001D6E09F
:105FD7003EF09001D3E004F0229001D3E0FFEFB44C
:105FE70006389001D6E0FEA3E0FFEFC4F8540FC8CF
:105FF70068FFEEC454F048FE9001D6EEF0A3EFF030
:10600700AF56128A0D7E009001D7E02FF09001D68F
:10601700E03EF09001D3E004F0229001D3E0FFEFDF
:10602700B407459001D6E0FEA3E0FFEFC4F8540F94
:10603700C868FFEEC454F048FE9001D6EEF0A3EF17
:10604700F0AF56128A0D7E009001D7E02FF0900135
:10605700D6E03EF09001DBE0FF9001D3EFF0900136
:09606700DAE0FF9001D2EFF02213
:106070009001D3E0FFEF70279001E0E4F0A3E4F09B
:106080009001D6E0FEA3E0FF9001D8EEF0A3EFF080
:106090009001DEE4F0A3E4F09001D3E004F02220CC
:1060A00061030262469001D3E0FFEFB4010EAF56E8
:1060B000128A0D8F7A9001D3E004F0229001D3E090
:1060C000FFEF6402706CE57AC454F0F57AAF5612B3
:1060D0008A0DEF257AF57A9001E0E0FEA3E0FF74E7
:1060E000002FF58274083EF583E57AF0AF7A7E00E2
:1060F0009001DFE02FF09001DEE03EF09001E1E062
:1061000004F070069001E0E004F09001D9E024FF73
:10611000F09001D8E034FFF09001D8E0FEA3E0FF5A
:10612000EF4E60079001D37401F0229001D3E00498
:10613000F0229001D3E0FFEFB40316AF56128A0DA0
:106140007E009001DCEEF0A3EFF09001D3E004F0CC
:10615000229001D3E0FFEFB404389001DCE0FEA30D
:10616000E0FFEFC4F8540FC868FFEEC454F048FED7
:106170009001DCEEF0A3EFF0AF56128A0D7E009096
:1061800001DDE02FF09001DCE03EF09001D3E0046F
:10619000F0229001D3E0FFEFB405389001DCE0FE7F
:1061A000A3E0FFEFC4F8540FC868FFEEC454F048F2
:1061B000FE9001DCEEF0A3EFF0AF56128A0D7E00E8
:1061C0009001DDE02FF09001DCE03EF09001D3E0A3
:1061D00004F0229001D3E0FFEF640670699001DCC7
:1061E000E0FEA3E0FFEFC4F8540FC868FFEEC4540C
:1061F000F048FE9001DCEEF0A3EFF0AF56128A0DEE
:106200007E009001DDE02FF09001DCE03EF0900197
:10621000DCE0FEA3E0FF9001DEE0FCA3E0FDEDB5D5
:10622000071AECB506169001DAE0FF9001D2EFF004
:106230009001DBE0FF9001D3EFF022227F021200F9
:07624000869001D2E4F02278
:108A0D008F78E578B430037F0022E578B431037FA9
:108A1D000122E578B432037F0222E578B433037F77
:108A2D000322E578B434037F0422E578B435037F5F
:108A3D000522E578B436037F0622E578B437037F47
:108A4D000722E578B438037F0822E578B439037F2F
:108A5D000922E578B441037F0A22E578B442037F09
:108A6D000B22E578B443037F0C22E578B444037FF1
:108A7D000D22E578B445037F0E22E578B446037FD9
:078A8D000F22D2637F0022DB
:0B0086008F79758400857999D2622281
:109B4500C2B5900003741EF0900003E0FFEF6004BF
:079B5500C2B580F4D2B52275
:105C970000000000000004000000080000000C00E5
:105CA70000001000000014000000180000001C0095
:105CB70000002000000024000000280000002C0045
:105CC70000003000000034000000380000003C00F5
:105CD70000004000000044000000480000004C00A5
:105CE70000005000000054000000580000005C0055
:105CF70000006000000064000000680000006C0005
:105D070000007000000074000000780000007C00B4
:105D170000108000001084000010880000108C0024
:105D270000109000001094000010980000109C00D4
:105D37000010A0000010A4000010A8000010AC0084
:105D47000010B0000010B4000010B8000010BC0034
:105D57000010C0000010C4000010C8000010CC00E4
:105D67000010D0000010D4000010D8000010DC0094
:105D77000010E0000010E4000010E8000010EC0044
:105D87000010F0000010F4000010F8000010FC00F4
:105D970000218000002184000021880000218C0060
:105DA70000219000002194000021980000219C0010
:105DB7000021A0000021A4000021A8000021AC00C0
:105DC7000021B0000021B4000021B8000021BC0070
:105DD7000021C0000021C4000021C8000021CC0020
:105DE7000021D0000021D4000021D8000021DC00D0
:105DF7000021E0000021E4000021E8000021EC0080
:105E07000021F0000021F4000021F8000021FC002F
:105E170000318000003184000031880000318C009F
:105E270000319000003194000031980000319C004F
:105E37000031A0000031A4000031A8000031AC00FF
:105E47000031B0000031B4000031B8000031BC00AF
:105E57000031C0000031C4000031C8000031CC005F
:105E67000031D0000031D4000031D8000031DC000F
:105E77000031E0000031E4000031E8000031EC00BF
:105E87000031F0000031F4000031F8000031FC006F
:1041EE009001ADE0FFEF70769001BFE0FFEFD3944A
:1041FE00034003024652206003024652C260900101
:10420E00BCE51EF0A3E51FF09001BCE0FEA3E0FFAD
:10421E00EE541FFE9001B6EEF0A3EFF09001BCE05D
:10422E00FEA3E0FFEEC4135407FF7E009001BCEE28
:10423E00F0A3EFF09001BDE0FF9001AFEFF0900121
:10424E00AEE4F09001BCE0FEA3E0FFEF4E7004D2AE
:10425E005E22229001BDE0FF9001ADEFF0229001B1
:10426E00ADE0FFEFB4011A2060030246529001B890
:10427E00E51EF0A3E51FF0C260D25E9001ADE4F042
:10428E00229001ADE0FFEF64027040206003024611
:10429E0052C2609001AEE0FFEF70119001B8E51EC2
:1042AE00F0A3E51FF09001AEE004F0229001AEE025
:1042BE00FFEF640160030246529001BAE51EF0A3BF
:1042CE00E51FF0D25E9001ADE4F0229001ADE0FF6B
:1042DE00EF640360030243FF206003024652900125
:1042EE00A7740AF0C2609001AEE0FFEF7029900152
:1042FE00B8E51EF0A3E51FF09001B4E4F0A3E4F0DE
:10430E009001B0E4F0A3E4F09001B2E4F0A3E4F085
:10431E009001AEE004F0229001AEE0FFEF64017078
:10432E00799001BCE51EF0A3E51FF09001BCE0FE04
:10433E00A3E0FF9001B1E02FF09001B0E03EF090CD
:10434E0001BCE0FCA3E0FD9001B2E475F001128621
:10435E0057AFF0FEEF25E0FFEE33FE74002FF5822F
:10436E0074043EF583ECF0A3EDF09001B5E004F09B
:10437E0070069001B4E004F09001B6E0FEA3E0FFF9
:10438E009001B4E0FCA3E0FDED6F7002EC6E6003F3
:10439E000246529001AE7402F0229001AEE0FFEFA1
:1043AE00640260030246529001BAE51EF0A3E51FB7
:1043BE00F09001ADE4F09001B0E0FEA3E0FF9001BB
:1043CE00BAE0FCA3E0FDEDB5071FECB5061B9001AE
:1043DE00B6E0FEA3E0FF9001B8E0FCA3E0FD129969
:1043EE00167F007E90129B84227F017E90129B840A
:1043FE00229001ADE0FFEF640460030245302060BF
:10440E00030246529001A7740AF0C2609001AEE01A
:10441E00FFEF70299001B8E51EF0A3E51FF09001A3
:10442E00B4E4F0A3E4F09001B0E4F0A3E4F0900162
:10443E00B2E4F0A3E4F09001AEE004F0229001AEFD
:10444E00E0FFEF640170739001BCE51EF0A3E51F61
:10445E00F09001BCE0FEA3E0FF9001B1E02FF090E0
:10446E0001B0E03EF09001BCE0FCA3E0FD9001B293
:10447E00E475F001128657AFF0FEEF25E0FFEE3344
:10448E00FE74002FF58274043EF583ECF0A3EDF07C
:10449E009001B5E004F070069001B4E004F09001D4
:1044AE00B4E0FEA3E0FFEF64007003EE640260036D
:1044BE000246529001AEE004F0229001AEE0FFEF12
:1044CE0064026003024652755B559001BAE51EF018
:1044DE00A3E51FF09001B0E0FEA3E0FF9001BAE06B
:1044EE00FCA3E0FDEDB50727ECB506239001B6E081
:1044FE00FEA3E0FF1280107F007E90129B8490013D
:10450E00B8E0FEA3E0FFEF4E6012755CAA800D7559
:10451E005B00755C007F017E90129B849001ADE480
:10452E00F0229001ADE0FFEF6405600302463D20EE
:10453E0060030246529001A7740AF0C2609001AE69
:10454E00E0FFEF70299001B8E51EF0A3E51FF09093
:10455E0001B4E4F0A3E4F09001B0E4F0A3E4F09031
:10456E0001B2E4F0A3E4F09001AEE004F022900179
:10457E00AEE0FFEF640170769001BCE51EF0A3E59E
:10458E001FF09001BCE0FEA3E0FF9001B1E02FF020
:10459E009001B0E03EF09001BCE0FCA3E0FD900184
:1045AE00B2E475F001128657AFF0FEEF25E0FFEE94
:1045BE0033FE74002FF58274043EF583ECF0A3ED08
:1045CE00F09001B5E004F070069001B4E004F090B4
:1045DE0001B6E0FEA3E0FF9001B4E0FCA3E0FDED28
:1045EE006F7002EC6E705D9001AEE004F0229001EF
:1045FE00AEE0FFEF6402704C9001BAE51EF0A3E549
:10460E001FF09001ADE4F09001B0E0FEA3E0FF904A
:10461E0001BAE0FCA3E0FDEDB5070CECB506087F92
:10462E00007E90129B84227F017E90129B842290AA
:10463E0001ADE0FFEFD39405400A9001ADE4F09098
:05464E0001AEE4F022C2
:103286009001BFE0FFEF702A9001ADE0FFEFD3940D
:103296000240030237ED305F030237ED205D030283
:1032A60037ED9001BEE0FF9001BFEFF09001C0E462
:1032B600F0229001BFE0FFEFB401179001C2E0FEDB
:1032C600A3E0FFEE4420FE129B84C25D9001BFE4A2
:1032D600F0229001BFE0FFEF640270489001C0E069
:1032E600FFEF7019205F169001C2E0FEA3E0FFEE2B
:1032F6004440FE129B849001C0E004F0229001C07D
:10330600E0FFEFB4011E305F030237ED9001C4E029
:10331600FEA3E0FF129B84C25D9001BFE4F0900122
:10332600C0E4F0229001BFE0FFEF6403706C9001EF
:10333600C0E0FFEF701C305F030237ED9001C2E082
:10334600FEA3E0FFEE4460FE129B849001C0E00401
:10335600F0229001C0E0FFEFB40118305F0302379E
:10336600ED9001C4E0FEA3E0FF129B849001C0E053
:1033760004F0229001C0E0FFEFB4021E305F0302AA
:1033860037ED9001C6E0FEA3E0FF129B84C25D907C
:1033960001BFE4F09001C0E4F0229001BFE0FFEF2E
:1033A600640460030235369001C0E0FFEF7033908D
:1033B60001C2E0FEA3E0FF9001C4E0FCA3E0FD1221
:1033C60092F59001CAE4F0A3E4F09001CCE4F0A3F6
:1033D6007480F09001C8E4F0A3E4F09001C0E0042A
:1033E600F0229001C0E0FFEFB4011C305F0302370A
:1033F600ED9001C2E0FEA3E0FFEE4480FE129B8446
:103406009001C0E004F0229001C0E0FFEFB4021882
:10341600305F030237ED9001C4E0FEA3E0FF129B8C
:10342600849001C0E004F0229001C0E0FFEF640345
:103436007063305F030237ED9001C8E475F0011246
:103446008657AFF0FEEF25E0FFEE33FE74002FF552
:103456008274043EF583E0F56AA3E0F56BAF6BAECC
:103466006A129B849001CBE0256BF09001CAE0358F
:103476006AF09001CDE024FFF09001CCE034FFF03B
:103486009001CCE0FEA3E0FFEF4E60022222900105
:10349600C0E004F0229001C0E0FFEFB4041E305FEC
:1034A600030237ED9001CAE0FEA3E0FF129B849071
:1034B60001C17464F09001C0E004F0229001C0E004
:1034C600FFEF6405706A9001C1E0FFEF701990018B
:1034D600CFE004F070069001CEE004F09001BFE466
:1034E600F09001C0E4F022306046C260851E6C8513
:1034F6001F6D9001C0E4F0E56DB40011E56CB49069
:103506000C9001BFE4F09001C0E4F0C25DE56D648B
:10351600017004E56C649060030237ED9001C0E42D
:10352600F09001CFE004F070069001CEE004F022A6
:103536009001BFE0FFEF640560030237ED9001C024
:10354600E0FFEF702B9001CAE4F0A3E4F09001CC09
:103556007402F0A3E4F09001C8E4F0A3E4F0900153
:10356600C2E0FEA3E0FF128C9E9001C0E004F022B0
:103576009001C0E0FFEFB4011C305F030237ED900D
:1035860001C2E0FEA3E0FFEE44A0FE129B84900180
:10359600C0E004F0229001C0E0FFEF6402706330E7
:1035A6005F030237ED9001C8E475F001128657AF4C
:1035B600F0FEEF25E0FFEE33FE74002FF582740473
:1035C6003EF583E0F56AA3E0F56BAF6BAE6A129B3E
:1035D600849001CBE0256BF09001CAE0356AF0904B
:1035E60001CDE024FFF09001CCE034FFF09001CC57
:1035F600E0FEA3E0FFEF4E600222229001C0E0044D
:10360600F0229001C0E0FFEFB4031E305F030237E3
:10361600ED9001CAE0FEA3E0FF129B849001C17405
:1036260064F09001C0E004F0229001C0E0FFEF6476
:103636000470659001C1E0FFEF70149001CFE004C3
:10364600F070069001CEE004F09001C0E4F0223064
:103656006046C260851E6C851F6D9001C0E4F0E572
:103666006DB40011E56CB4900C9001BFE4F09001CC
:10367600C0E4F0C25DE56D64017004E56C649060C1
:10368600030237ED9001CFE004F070069001CEE022
:1036960004F09001C0E4F0229001C0E0FFEF70203A
:1036A6009001CAE4F0A3E4F09001CC7402F0A3E424
:1036B600F09001C8E4F0A3E4F09001C0E004F02229
:1036C6009001C0E0FFEFB4011C305F030237ED90BC
:1036D60001C2E0FEA3E0FFEE44C0FE129B8490010F
:1036E600C0E004F0229001C0E0FFEF640270633096
:1036F6005F030237ED9001C8E475F001128657AFFB
:10370600F0FEEF25E0FFEE33FE74002FF582740421
:103716003EF583E0F56AA3E0F56BAF6BAE6A129BEC
:10372600849001CBE0256BF09001CAE0356AF090F9
:1037360001CDE024FFF09001CCE034FFF09001CC05
:10374600E0FEA3E0FFEF4E600222229001C0E004FB
:10375600F0229001C0E0FFEFB4031E305F03023792
:10376600ED9001CAE0FEA3E0FF129B849001C0E049
:1037760004F09001C17464F0229001C0E0FFEF6490
:103786000470649001C1E0FFEF70199001CFE0046E
:10379600F070069001CEE004F09001C0E4F09001D4
:1037A600BFE4F022306040C260851E6C851F6D90BC
:1037B60001C0E4F0E56DB40011E56CB4900C900125
:1037C600BFE4F09001C0E4F0C25DE56DB40118E518
:1037D6006CB490139001C0E4F09001CFE004F07057
:0737E600069001CEE004F0A3
:0137ED0022B9
:048010008E0F8F1030
:10801400D3E510947DE50F940040047F0180027F36
:1080240000C3E510943FE50F940050047E018002E4
:108034007E00EE4FFFEF600302810CE510AE0F7877
:1080440002C333CE33CED8F9FF74992FF582745C12
:108054003EF583E493F511740193F512E510AE0F28
:108064007802C333CE33CED8F9FF74972FF58274D8
:108074005C3EF583E493FE740193FF8F179001AD8A
:10808400E0FFEF6405FF9001E8EFF09001AEE0FF40
:10809400EF6401FF9001E9EFF0AD12AC11AF1712DC
:1080A400963F9001ADE0FFEF6405FF9001E8EFF02B
:1080B4009001AEE0FFEF6403FF9001E9EFF0751566
:1080C40000751600C3E51594045033AE15AF16744D
:1080D400002FF58274043EF583E0FF7E008E138F3B
:1080E40014AB14AD12AC11AF171294710512E51252
:1080F400700205110516E5167002051580C690017B
:08810400E8E4F09001E9E4F069
:01810C002250
:109916008E6E8F6F8C708D717B017A047900AC022C
:10992600AD01AF71AE7012752EE5712480FFE57042
:109936003400FE7B017A047980AC02AD0112752EEB
:0199460022FE
:048C9E008E5D8F5EFA
:108CA200E55EAE5D7802C333CE33CED8F9FF749958
:108CB2002FF582745C3EF583E493F55F740193F5BE
:108CC20060E55EAE5D7802C333CE33CED8F9FF7471
:108CD200972FF582745C3EF583E493FE740193FF53
:108CE2008F63756100756200C3E5619404502BAD1A
:108CF20060AC5FAF63129A63AC61AD6274002DF534
:108D02008274043CF583EFF00560E5607002055F54
:0A8D12000562E5627002056180CE83
:018D1C002234
:0892F5008E648F658C668D67A5
:1092FD00756800756900E5652401FFE5643400FEBD
:10930D00EF25E0FFEE33FEC3E5699FE5689E50292A
:10931D000567E567AE667002056614FF1274D7AC7B
:10932D0068AD6974002DF58274043CF583EFF0058A
:09933D0069E5697002056880BD54
:019346002204
:109B84008E188F19205FFD851825851926755A00B2
:039B9400D25F227B
:10770F00205E030278499001AFE0FFEF600302773C
:10771F00D6C25E9001B6E0FEA3E0FFEFB4FF0BEE22
:10772F00B41F0775840075EF03229001B6E0FEA326
:10773F00E0FFEEFF7E008F769001B7E0FFEF54FF82
:10774F00F577E576700B7FFF8F779001E57401F089
:10775F0022E576B41516C3E577648094B3500D9087
:10776F0001E27401F09001E4E577F022E576B416BA
:10777F0016C3E577648094F2500D9001E27402F025
:10778F009001E4E577F022D3E5766480948040376A
:10779F00C3E57664809495502ED3E577648094800A
:1077AF004025AF77EF3395E0FEC3EF94FBEE648097
:1077BF00948050139001E27403F09001E3E576F0AA
:1077CF009001E4E577F0229001AFE0FFEF640270E3
:1077DF00699001B6E0FEA3E0FFEF64014E702B90BD
:1077EF0001BFE0FFEF70F89001C2E4F0A3747FF0E7
:1077FF009001BAE0FEA3E0FF9001C4EEF0A3EFF01A
:10780F009001BE7404F0D25DC25E9001B6E0FEA39B
:10781F00E0FFEF64024E70229001BFE0FFEF70F8BF
:10782F009001BAE0FEA3E0FF9001C2EEF0A3EFF0EB
:0A783F009001BE7405F0D25DC25E38
:01784900221C
:10FC0000C2AF12FCD812FD10E4F550F551E42551B5
:10FC1000FFE5503480FE12FCB6AD07AF51AE501276
:10FC2000FC5F0551E55170020550C3E550948040DA
:10FC3000DC755080755100AF51AE5012FCC7AD0756
:10FC4000AF51AE5012FC8A0551E55170020550C308
:10FC5000E55094F440E1D2AF75840075EF0122C203
:10FC6000AF75840F53A1FEE4F5B1F58443B701F5F8
:10FC700084438F018E088F098F828E83EDF0E4F527
:10FC800084538FFEF58453B7FE22C2AF75840F53A1
:10FC9000A1FE75B110E4F58443B701F584438F01EB
:10FCA0008E088F098F828E83EDF0E4F584538FFEEA
:10FCB000F58453B7FE22C2AF75B1218E0A8F0B8F28
:10FCC000828E83E493FF22C2AF75B1318E0A8F0B0F
:10FCD0008F828E83E493FF22C2AFE4FFFEE4F5B18E
:10FCE000F58443B701F584758F03AD07AC068C0826
:10FCF0008D098D828C83F0F58FF58453B7FE2FFF2D
:10FD000074043EFEC3948040D4E4F58453B7FE22CD
:10FD1000C2AF7F007E8075B110E4F58443B701F572
:04FD200084758F0354
:10FD2400AD07AC068C088D098D828C83F0F58FF5B8
:10FD34008453B7FE2FFF74043EFEC3648094744062
:08FD4400D1E4F58453B7FE225F
:0300000002007685
:0C007600787FE4F6D8FD7581A002624797
:1085ED00BB010689828A83E0225002E722BBFE028C
:0985FD00E32289828A83E49322BF
:10860600BB010CE58229F582E5833AF583E0225029
:1086160006E92582F8E622BBFE06E92582F8E22273
:0D862600E58229F582E5833AF583E493228D
:10863300BB010689828A83F0225002F722BBFE0126
:02864300F32220
:10864500EF8DF0A4A8F0CF8CF0A428CE8DF0A42E49
:02865500FE2203
:10865700A3F8E0C5F025F0F0E582158270021583D6
:06866700E0C838F0E82233
:10866D00D083D082F8E4937012740193700DA3A39C
:10867D0093F8740193F5828883E4737402936860B0
:06868D00EFA3A3A380DFB0
:00000001FF
